:020000041100E9
:10300000002373B52B4D2C4C28006361022601F080
:103010006FF94021FE2221742800284B009601F010
:10302000B9F9002836D1217CFF222800244B0096D4
:1030300001F0B0F900282DD1224BA2899A4226D165
:10304000E389214A93420DD1204B6361204B2268D2
:10305000002A03D1002B01D043CB43C4280001F048
:1030600085F973BD1B4A934201D00023EFE71A4B49
:103070001A4A1B68934206D9C02304222800217CE7
:103080009B0001F0FDF9114B6361154BDFE7002355
:103090002374EAE7CC233821AC2228009B01217459
:1030A00001F0EEF90028F2D10E4B63610E4BE38183
:1030B0000E4BCCE7F441FF1FA461FF1FB061FF1F5F
:1030C000B261FF1F59590000830500001D41001126
:1030D00048BD001182150000C861FF1F8713000062
:1030E00054BD0011D5410011AAAAFFFF3CBD00113B
:1030F000F7B5164B0192C318021D002000938823D8
:103100005B05D3181B685C1C1AD09CB2402C18D8E5
:103110008D781E0CAC466746CD782D023D43AE42FD
:1031200006D1019800280ED110000C70240A4C70B2
:1031300003249BB20733A343D218009B9A42DED3E9
:10314000FEBD4432F9E71000FAE7C046FC0F00006C
:10315000802213B503000324019189B25201073183
:103160009B18A14304305A1A88235B05C3181B68B7
:10317000591C03D190429241104016BD99B240298A
:1031800007D80B000733A343C0189042ECD30020AC
:10319000F3E74430F9E7134B134A1B68126810B584
:1031A000FA24934201D81A00F824104BE4021B6859
:1031B0009A4210D813000E4A12689A420ED3013375
:1031C00007D1F823DB029C4203D10A49054808F0E5
:1031D0002FFD200010BDFC24E402ECE7FE24E402F5
:1031E000F7E7C04600C0071100D0071100E0071143
:1031F00000F00711FFFFFF7FF0B59BB015000490B2
:103200000391402A00D9A0E006AB59801A80FFF74D
:10321000C2FF0400042816D9002206A9FFF768FFA0
:10322000052810D906AB1B88AB420CD1002D07D066
:10323000514B2A000499C01808F0FAFB002802D16B
:1032400001201BB0F0BD06AB1D8020000699FFF7E2
:103250007FFF041E7BD1069B0793FFF79CFF802313
:103260005B01C618802307001B039E4201D3F8268A
:10327000F60288235B05F31801931B68013302D023
:10328000019808F0DDFA3D49019808F0D1FC3B1D9A
:103290000293331D05938822029B52059B181B68DD
:1032A00008935A1C3CD044219AB20091402A04D879
:1032B0000320D11D814389B2009103991B0C8B42DD
:1032C00024D0402A22D80122300008A9FFF710FF9D
:1032D000021E1BD1380008A9FFF70AFF04000428CA
:1032E00031D9009A059B9B1880225201B218934253
:1032F00040D288235B05C118009A09A808F0F8FBA2
:103300001D4B009A09A9F01808F072FC009A029B64
:103310009446634402931A4B029AFB189A42BAD31A
:1033200088235B05FC1821680198013908F080FCAE
:10333000200008F085FA039A07AB5A8030000799FD
:10334000FFF706FF0400002C03D1002079E70428D2
:10335000FBD988235B05E018069908F069FC032374
:10336000EA1C9A4300D16BE7034B0499E01808F07C
:103370003FFC65E70424ECE704000011FFFFFF7F3A
:10338000F80F0000F7B505001400402A21D80027E7
:1033900001AE71803780FFF7FEFE042816D93A008F
:1033A0003100FFF7A5FE042810D93688BC420BD0A7
:1033B000BD4209D0221CB44200D9321C064B92B245
:1033C000C118280008F094FB30B2FEBDC04300B223
:1033D000FBE703204042F8E70400001137B5042260
:1033E00004000D0001A81649FFF7CCFF02000428D5
:1033F0000BD1019BA34208D3AB4204D0104901A8D2
:103400000195FFF7F9FE01203EBD0E4C2368200018
:10341000019308F015FA019920000139019108F093
:1034200007FC80235B01E418074B9C42EED1042289
:10343000034901A80195FFF7DFFE0020E4E7C0463D
:103440005555000000C007110000081130B589B0C3
:1034500008F02EFA10226946254808F061F9254B3C
:10346000009A9A420ED1019B029A0F2B33D8002169
:1034700001240698013B08D2002900D00292029B49
:10348000013331D10023029325E0551CF2D1020013
:103490002100EFE710341022200004A908F040F9C1
:1034A000029B013301D1069B0293882304995B059B
:1034B000C918059B06981A03120B049105928142C4
:1034C00003D02B4201D108F013FB019B013B019378
:1034D000019B002BDED1029B002B03D004930498A8
:1034E0004168084709B030BDE025014C2D03EFE7E6
:1034F00000000111504859368022F8B5964C974B80
:10350000D200002120001C6008F0B2F92300944A88
:1035100088331A60934B1A786A23002A00D011333B
:10352000E3620A232365904B37221B780820A363AC
:103530008E4B2118E361102323628D4B3B25636181
:10354000C823DB00A36123008C331A602823013ACF
:10355000E26320646364CA67043A211DCA672100DC
:10356000BC310D602100C03108602100C4310B6006
:1035700021000635CC310D602100083DC8310D60B9
:103580002100D0310A602200D43210602200D832EB
:10359000136022000227E032210017604222DC3152
:1035A0000A6021001B3DE4310D602100E831086014
:1035B0002100EC310B6023000521F4331960230056
:1035C000F0331A602300183290331A6023009433CA
:1035D000186023001E3A98331A60AF23DB00236083
:1035E000644BFA262363644B644DE360644BF03113
:1035F000A3642300FF31FC33B600A16021611E608B
:10360000A5627325E5656D3D6565A56596255D4AF1
:10361000AD00E264666258606766A566002709250A
:10362000A767E566584F594D606720002567E26738
:103630003A6015279C30676007001A203860200028
:10364000A0300700212038602000A83007004C4837
:1036500038602000F830066026006427A436376002
:1036600026005F3FAC3637602600033FB036376038
:103670002600C637B436376026000027B8363760D4
:1036800038269E60424E96205E64424E5A66DE6147
:10369000414E9A645E62F53EFF3E9E621E269A6728
:1036A000354A8000DE661F675F67DD651D6618624C
:1036B000DA67BE23394A5B00E250394BD8382350D1
:1036C00004302250C4225200A350C623E4205B00E1
:1036D000E1500433334AE1503349344BD16034492B
:1036E000800019503349E938FF3819503249043005
:1036F000195032493248D16132491163324951631C
:103700001900F4310860CE20304940001160304982
:10371000195019002F48F83108602F49D1658221CE
:103720002E4A89005A501A002D490832D1671A00D2
:103730002C49B432116088212B4A89005A501A0052
:103740002A49883211602A4ADA6408F0E9F801202F
:1037500007F08EFFF8BDC0460004FF1F4064FF1F46
:10376000206FFF1F3844FF1F4A0AFF1F3A0700005F
:1037700080C3C9019A020000DC0500006A1800003D
:1037800050C3000088130000F009FF1F204E000006
:103790006509FF1F68100000C409000040420F00C7
:1037A00010270000FC00FF1FC11BFF1F0000FF1FB0
:1037B000152CFF1FA52FFF1F3D2EFF1F811FFF1F71
:1037C0007126FF1F9D1FFF1F4921FF1F0D1FFF1F98
:1037D0009528FF1F7D29FF1FD918FF1FA127FF1F55
:1037E000C524FF1FD124FF1F0D1EFF1FC51EFF1F75
:1037F000851DFF1F0223F0B50124614D614E2B7022
:10380000614B91B01C70614F039333680021082015
:10381000FB7006F0EFFD082006F0E6FC002398425E
:1038200005D0FA78552A02D0332A00D09BE03360C5
:10383000042006F059FF07F0F3FFFFF75DFE07F0E5
:103840003FFF1F2201240021514B10AE1A70514B33
:103850001C70514B1970514B19689143163A0A4329
:103860001A60602219689143403A0A431A6007F0CF
:10387000D7FE07F00DFFC120FF21494B80001A58E9
:103880008A431A50C522920098588843BF39014391
:1038900099509858434908408021C901014380202C
:1038A00099509958C0050902090A0143995080218D
:1038B0003D48490108F084F8032322003B49019464
:1038C00000933B4808F0FCF82C223A4905A808F080
:1038D0000FF905AC61782078023406F0A5FCA64209
:1038E000F8D1354C0020012106F0B2FD2268334B9F
:1038F00003201A40A023DB021343236080232268A5
:103900009B041343236022682D4B1A4080239B03A2
:10391000134323602B4A2C4B934200D8012007F01D
:1039200017FF08F08DF880232268DB04134323601F
:10393000287808F015F9039B1878C0B208F038F819
:1039400008F0E6F82149042008F022F806F098FE75
:1039500000F0A8F800F0EAFD00F092FE00F00CFA8A
:10396000002011B0F0BD00932100184A042007F098
:10397000CFFF8023DB059C62FFF768FD58E7C04658
:103980004A0AFF1F34F000403844FF1FD461FF1F74
:10399000480AFF1F490AFF1F680AFF1FBCF00040CA
:1039A00000E100E0FF00FFFF3C44FF1FC056FF1F87
:1039B0003C54FF1F60BC001114F00040FF7FF8FF73
:1039C000FFFF9FFF0080FF1F206FFF1F3B000108CC
:1039D00070B500252549264A26484D6308CA1B05AF
:1039E0001B0DED188242F9D100268022224B920550
:1039F0008B630921214B224C1E62224B1120DA6776
:103A0000214BDA688A43DA609A6820490A409A6052
:103A1000266008F005F9112007F022FF8022636C70
:103A200093436364EE24E4006C43194A200C0400C1
:103A3000642390420AD8FA223300D200904205D97A
:103A4000144B0A21C01807F0ABFEC3B2124A112072
:103A50001372D48007F014FF104B1B78002B04D195
:103A60000F4B1021187807F0F3FF70BD00000540E0
:103A70008805054000060540FF01000000F00040F9
:103A80000038004004E100E03CF00040FFDFFFFFB1
:103A9000B70B000030F8FFFFBC61FF1FF663FF1F8C
:103AA000F461FF1F002210B51100112007F0A8FEDD
:103AB00010BD0000F8B500230926374F374C3B6294
:103AC000E3681120B343E36007F0CAFE112008F059
:103AD000A7F8112007F0C4FD402322688025134376
:103AE000236080236268DB0213436360A3682C4A6F
:103AF0002B43A360A36802211340A3608023A26824
:103B00009B0113431022A360236C0720934323647B
:103B1000236C0F3A1343236480235B003B62226BC8
:103B2000204B1A402263626B1A406263A26B1A40F8
:103B3000A263E26B1340E363E3681B4A1340E36054
:103B400006F072FB0121072006F082FC174B1120C2
:103B50005A6C15435D6407F00BFEFD21144B154AAA
:103B600089005A508023C720626B5B031343636351
:103B7000E36880003343E3600F4B104A195811404B
:103B8000802212020A431A50802292051A600822EB
:103B90000B4B5A63F8BDC04600F000403CF00040BB
:103BA000FFFFDFFFEFFFEFFFFFFF7FFF0038004069
:103BB0000000FF1FD139001100E100E0FF00FFFF0E
:103BC0000000054030B503A804880B20002C0ED15E
:103BD0004968074D08784978090201430A20A9423B
:103BE00005D1012120001980024B1B7A137030BDD2
:103BF000192A0000BC61FF1FF7B5150008AA168836
:103C00004A680F4F14785278120222430A24BA42AB
:103C100014D10122DBB2019200962A0007F080FC49
:103C2000041E0BD1074B1B68002B07D068782A783D
:103C30000002104342425041013098472000FEBD2F
:103C4000022900004061FF1F30B5012503790400FF
:103C5000BFB02B4211D00A49408806F0CDFF284260
:103C60000BD0084B01A95B8D4D800B80064B0022C9
:103C70001B7A60880B7104F09FF83FB030BDC046DE
:103C80003861FF1F6840FF1FBC61FF1F10B5054969
:103C9000054806F067FF0421044A054806F024FFA2
:103CA00010BDC0463861FF1FFFFF00008CBC001133
:103CB0006840FF1F10B5024804F000FF10BDC04669
:103CC000493C0011062310B5837010330371443B47
:103CD00043712A3383714433C371002302220121CB
:103CE00003720E4B027041701C8881724472197A03
:103CF0000273C1729A784273DA7882730322C273B4
:103D00001A7902745A7942740C2282749A79C274B4
:103D1000DB7903751123C370152010BDBC61FF1F33
:103D200010B5142007F01CFE124B1422002118605D
:103D300007F09EFD002007F003FE012007F0F8FDCC
:103D4000022007F0CDFD032004F05CF9042006F00A
:103D500071F9052003F09AFB062004F067F80720AC
:103D600001F05AFA082006F09FFE092001F034F80D
:103D700010BDC0464461FF1F07F032FE012007F06E
:103D800027FD07F095FE0000094B10B5040098428E
:103D900005D0012904D12000064906F0E3FE10BD3C
:103DA0000229FCD1013904F047FE0028F3D0F6E7E0
:103DB000FEFF00006A61FF1F70B50D7A100004AAB3
:103DC0002C00168810221440154220D1002E20D13C
:103DD0000A78022A18D14A68517815780E4A0902E1
:103DE0002943914205D00D4A914209D01C800A24F2
:103DF00004E014220A491A8007F07AFE200070BD00
:103E00000C2208491A80F7E71C800124F6E70824F1
:103E1000F4E70B24F2E7C046F3FF0000F4FF0000D4
:103E2000C442FF1F6CBD001110B5040007490848CB
:103E300006F098FE074804F081FD0020E40704D551
:103E40000721054A054806F04FFE10BD6A61FF1FB5
:103E5000FFFF0000893D0011D0BC0011AC40FF1FE6
:103E600000B50C4BBFB01A780B4902A800F0C2FC99
:103E70006B4680B2D880002809D06A46074B01A95A
:103E80001B889380064B0022188803F095FF3FB0F3
:103E900000BDC0464861FF1F4961FF1F0641FF1F6B
:103EA0001042FF1F00B50C4BBFB01A780B4902A897
:103EB00001F0C8FE6B4680B2D880002809D06A465F
:103EC000074B01A95B8D9380064B0022188803F0F5
:103ED00073FF3FB000BDC0467261FF1F7361FF1FDB
:103EE000AC40FF1F1042FF1FF7B50E00377A1C00D1
:103EF00008AB11003D001A8820231D401F423CD111
:103F00003378022B3BD173681F785B781B023B43ED
:103F10001E4FBB4208D01E4FBB4214D01D4DAB42BA
:103F200021D00A252800FEBD002A2AD1142C2AD827
:103F30002200F06807F0DCFD174B1C70012CF1D952
:103F4000FFF7B0FFEEE7002A1BD1202C1BD8220080
:103F5000F06807F0CDFD114B04211C70104B187850
:103F600007F076FDDEE7E3B20124009201940A0037
:103F7000310007F0D5FA0500D4E70825D2E701257E
:103F8000D0E70B25CEE70D25CCE7C046F3FF0000B8
:103F9000F4FF0000022900007261FF1F4861FF1F4B
:103FA000F461FF1F332310B5040003700A22074990
:103FB000013007F09DFD064B0F201B681A0AE372C3
:103FC00022731A0C1B0E6273A37310BDBC61FF1F1A
:103FD000E461FF1F30B5012503790400BFB02B4217
:103FE00013D00B49408806F007FE28420DD06A46E0
:103FF000084B02A81B889380FFF7D4FF6B46D8803C
:104000000022608801A903F0D7FE3FB030BDC04652
:104010006A61FF1F0641FF1F10B5024804F04EFD04
:1040200010BDC046D53F001170B5160004AA148813
:1040300005AA15784A685078117800022A4A084380
:10404000801805284BD807F0EBFC03131E29343FDA
:104050000720042C0BD80522121BAA4200D92A00E3
:1040600022491A803000091907F042FD002070BD76
:104070000720112CFBD81222121BAA4200D92A00B9
:104080001B491A80EEE707200E2CF0D80F22121BD6
:10409000AA4200D92A0017491A80E3E70720032C17
:1040A000E5D80422121BAA4200D92A0012491A801C
:1040B000D8E70720032CDAD80422121BAA4200D921
:1040C0002A000E491A80CDE70720032CCFD80422FE
:1040D000121BAA4200D92A0009491A80C2E700220D
:1040E0000A201A80C3E7C046DCD5FFFF1BBD0011C4
:1040F0009061FF1F0BBD001106BD001101BD001135
:10410000FCBC001110B50D21024A034806F0ECFC7E
:1041100010BDC046F0BC00111C41FF1FF0B50024CB
:10412000274E85B03000B47100F0E2F8254D264BE3
:10413000EA89297C9A422FD10423300003AA00F097
:1041400057F90400300000F011F90123B371002C7D
:1041500034D16B4699892B68C9BA4B4329891B4ACC
:104160001B145B1853806B46D9896B6849BA89B2B6
:104170004B4369891B0C5B181548191C1BB2834201
:1041800000DD011C0B0400D5002113889180013350
:104190001380200005B0F0BD0227220003AB3000E1
:1041A000009700F0F7F80E230400297C012230006C
:1041B00000976B4400F0EEF80443C3E71C00E8E707
:1041C000F441FF1FA461FF1F83050000BC61FF1FB6
:1041D0000F27000073B5234E300000F089F8224D00
:1041E00007236A463000297C00F002F90400300001
:1041F000002C33D16B461B787F2B2FD800F0B6F8FC
:104200006B46D878F02302041B031A406B469B8848
:1042100016495BBA9BB21A432B68000953432A899B
:104220001B0C9B184B806B465A789B7812031B0122
:104230001A436B68024353436A891B0C9B180C4852
:104240001A1C1BB2834200DD021C130400D500229D
:104250000B888A8001330B80200076BD00F086F841
:104260000124F9E7F441FF1FA461FF1FBC61FF1F98
:104270000F27000070B5114C237C002B0FD0382B7A
:104280000ED10F4D280000F033F8CC23AC222800CB
:10429000217C9B0100F0F4F8280000F067F870BD65
:1042A000084BE2899A42FAD1054D280000F020F827
:1042B00000222800217C00F0C5F8EDE7A461FF1F73
:1042C000F441FF1F8305000010B5084B1A7C002A3B
:1042D00009D05B69002B06D09847041E01D0FEF779
:1042E0008FFE200010BD0124F9E7C046A461FF1F26
:1042F00070B5C17905000C00631E9C411A4BE402A5
:10430000E41849000460C9B2007906F0D7F8E979E9
:10431000687949000131C9B206F0D0F8E87909306E
:10432000C0B207F09DF90023E36661332360AA79E8
:104330005B3B002A0ED022689A43023B1343236062
:104340000A23E3610733236200232363A36301335A
:10435000E36370BD22689A4302231343236046231C
:1043600063610633A361EFE70050004070B500259C
:1043700004000368DD66C0790930C0B207F070FA46
:104380002900207906F036F82900607906F032F825
:1043900070BD0000F8B51E0006AB1D780023046850
:1043A0001700E366616007F083FA01238022E36669
:1043B0002B0027615200013B08D207F0B1FB082017
:1043C0000A4A1168002D03D12800F8BD2261F2E7E6
:1043D000236F034203D02369013D33700136136814
:1043E0005B1A032BEED90125EEE7C0466008FF1FDC
:1043F00070B51C00002305681600EB66696007F0C5
:1044000057FA01238022EB6623005200013B08D2B9
:1044100007F086FB08200A4A1168002C03D120000F
:1044200070BD2A61F2E72B6F034203D02B69013C78
:104430003370013613685B1A032BEED90124EEE7C3
:104440006008FF1F002370B504681500E366616013
:1044500007F02EFA0123E366256107F061FB802057
:10446000064A80001168636B034205D113685B1A2A
:10447000032BF8D9012070BD0020FCE76008FF1F66
:1044800070B51D00002304681600E366616007F044
:104490000FFA0123E36626610F33626B1A42FCD0E8
:1044A0002B0A23611023626B1A42FCD0EDB2256106
:1044B00007F036FB8020074A80001168636B0342D7
:1044C00005D113685B1A032BF8D9012070BD0020B9
:1044D000FCE7C0466008FF1F70B51E00002305689A
:1044E0001400EB66696007F0E3F90123A619EB6697
:1044F0000F33B4420ED107F013FB80200A4A80002C
:1045000011686B6B03420CD113685B1A032BF8D94B
:10451000012070BD21782961696B1942FCD00134FA
:10452000E7E70020F5E7C0466008FF1F10B5084C1C
:10453000E368002B08D18022064B52021B689B18AF
:104540006360054B1B68236007F012FBA06010BD81
:10455000E461FF1FC8F00040CCF0004070B5184A7D
:10456000936A916A9942FBD116498A689A421FD38D
:104570009A1A8B60144B0126186893B2D202D20E9D
:104580004343424300204C681B0A1B1912029B182C
:104590000E4C0A684B60551CA3420CD8002801D071
:1045A0004B600A600A4A136008680A4B186070BDC5
:1045B000581E821ADDE7084A30009B182A00EAE7F5
:1045C00000F00040E461FF1F140AFF1F40420F008B
:1045D000C8F00040CCF00040C0BDF0FF70B51F4CEB
:1045E00023793F2B01D93F2323711D4B22791A7068
:1045F0001878C0B207F0E4FA18231A491A4A0B8057
:104600001A4913800B805380A379194980200B80AD
:104610000C21938001334B43164D191C000183423A
:1046200000D9011C2980D1806379002B11D101337D
:104630006371237A012B01D8022323726279237AD2
:104640000D4853430A21584307F0AAF80B4D286040
:1046500070BDA02BEDD9A023EAE7C046D861FF1FAB
:10466000480AFF1F0E42FF1FE443FF1F0C42FF1FBB
:104670000A42FF1F0842FF1F71020000C861FF1FAE
:10468000F8B514210020FEF7A9FE114C011E114DB2
:1046900009D10C22104BC1CBC1C4280007F0E8F8A7
:1046A000FFF79CFFF8BD0C2220000C49FEF76AFEC4
:1046B0000C2802D0084B43CB43C40C2228000849E5
:1046C000FEF760FE0C28EBD00C220021E5E7C04687
:1046D000D861FF1FA461FF1F60BD0011FC0C00002A
:1046E000F50C0000F0B51D4C8022A5440400882084
:1046F00069465201400507F083FA902212016A448C
:104700001300200032C832C316C816C38023144CCD
:10471000144FA6689B033343A3603B6007F0F0F897
:104720008823A0685B05C01807F08AF80025882355
:1047300029008022A0685B05C01840196944520016
:1047400007F056FA80230135FF355B019D42EED11B
:10475000A6603E60044B9D44F0BDC046FCEFFFFFE9
:104760005443FF1F9808FF1F04100000F0B5040019
:1047700087B0002825D0684607F01AF81B4C02289D
:1047800006D106226946200007F052F9002816D00B
:104790006946002301250F262F00E25C0133100932
:1047A0001030874038002F00324097403A000243D3
:1047B0004A610439062BEFD16846FFF793FF07B033
:1047C000F0BD182269460A4807F01AFA6A46A300A3
:1047D000D358013305D01822FF21684607F048F866
:1047E000EAE70134062CF1D1E9E7C0466509FF1F6D
:1047F00000090011F0B5002504000E0085B0AA42A2
:1048000000D186E04B1C087801934B788978377982
:1048100009021943F3783F061B040B431F43039718
:1048200020706570252800D196E033D8112813D860
:1048300007F07EF969002501250125012501AA005F
:10484000B800B1002501250125012501250125011B
:104850002501250105011F01232800D1DEE0DB2809
:1048600000D02EE1042A00D8ACE01025052A05D09E
:10487000551F2A003800711D07F03AF90522310052
:10488000200007F035F92A003900601D07F030F9E3
:1048900005353EE0562859D010D8332800D19DE088
:1048A000552839D02628DAD19C4B2900132218002C
:1048B0001D0006F0DDFFFEF7A3FB5CE0712800D1D0
:1048C00077E0722800D180E0602800D18BE0DC28FE
:1048D000C5D1022A00D875E07378BFB26370B3788F
:1048E000A370032A05D0033A390092B2F01CFEF7F8
:1048F00083FC10223900E01CFEF744FDC51C002893
:1049000007DA60705CE00C222000854907F0F0F8BF
:104910000C25280005B0F0BD013A824D0C2A13D8B1
:10492000002A0AD02800019907F0E2F8FFF756FEA6
:104930000C2228007C49FEF75FFC29000C22601C39
:1049400007F0D6F80D25E4E70C22EBE7754D774B21
:104950002A0043CB43C2E9E7013A704D0C2A11D833
:10496000002A08D00199280007F0C2F80C2228007C
:104970006F49FEF741FC29001322601C07F0B8F8CC
:104980001425C6E70C22EDE705226A49601C07F0F2
:10499000AFF80625BDE712226749601C07F0A8F8AA
:1049A0001325B6E708226549601C07F0A1F8092520
:1049B000AFE77178F02905D8614B188801F09EFDAA
:1049C0000225A6E7FF236370FAE75E4B012A03D0B6
:1049D00072789A706270F3E79B78F4E72000FFF733
:1049E000E1FA050095E7013A564B574D062A10D8D3
:1049F000002A10D0012128005970019907F078F899
:104A000001F04EF829000622601C07F071F8072516
:104A10007FE70622EEE700225A70F3E7042A04D962
:104A20004A4D2F6007F0A4F8A860FFF797FD042215
:104A3000039003A9601C07F05BF8052569E7444D66
:104A4000062ADFD906222800019906F0F1FF002886
:104A5000D8D006220199280007F04AF806223D49DD
:104A60002800FEF7C9FB0123364A91780B43937067
:104A7000C8E7012AA6D07078FFF778FEA0E70128E2
:104A800000D0ECE6931E344F1A2B04D87378002B19
:104A900009D100F015F9314B39001D78601C6A1EF0
:104AA00007F026F835E7551E2A000199380007F06F
:104AB0001FF82B49AAB23800FEF79EFB00F036F92A
:104AC000E9E7DA281DD1042A00D87BE7082A15D99E
:104AD000B37972791B021343F27912041A43337AC1
:104AE0001B0613433B603B68052231002000039303
:104AF00006F0FEFF0422601D03A956E7FE23637043
:104B0000F1E7DE2800D05DE7511E012A01D1002522
:104B1000FFE6019800F0AAFFF9E7C046A461FF1F75
:104B20006CBD0011D861FF1FFC0C000060BD0011BE
:104B3000F50C0000B061FF1F9061FF1F5843FF1F7D
:104B40001042FF1FD461FF1FB442FF1FE461FF1F2B
:104B50006509FF1FADAC0000D563FF1FD363FF1FC6
:104B6000AEDE000070477047020010B5094B0A32F4
:104B7000094C92B2DA815A8298811882207802F028
:104B800023FB0422054B012120781A7006F060FFF8
:104B900010BDC046E242FF1F1E64FF1F1D64FF1FC1
:104BA000013870B5042809D806F03AFF030928082F
:104BB0001200234B0221187806F04AFF70BD204BEB
:104BC0000821187806F0BCFF00221E4B1A72F5E788
:104BD000802200241B4B1A4D52001A8108211A68AA
:104BE0002878DC7206F004FE2100287806F0D8FF51
:104BF000012000F073FE00F053FFDFE7104B0821A7
:104C0000187806F09DFF1048FFF75CF80F4B104A2C
:104C10009B79002093800F4A13808022094B520019
:104C2000D8721A8100F05AFE00F03AFF0A4B9B78C6
:104C3000002BC3D0094A136006F0D2FFBEE7C0467E
:104C4000F461FF1FC861FF1F1942FF1FD861FF1FDA
:104C5000E443FF1F0A42FF1FD461FF1F34F00040EE
:104C600010B501290BD1082809D1054B1B78002B61
:104C700005D02622034B04485A72FFF775FF10BD7A
:104C8000F663FF1FC861FF1FC40900000300F0B5F1
:104C90000A4D8E18B14202D152008018F0BD0C7836
:104CA0002F6824093C5D0F271C700C7801313C40B3
:104CB0002F683C5D5C700233ECE7C0460442FF1F86
:104CC0000E22114B10B51A700D23104C1049237091
:104CD000093A043B0F48637006F00AFF2D230122B6
:104CE0000D490E48E371FFF7D1FF01220C49FFF790
:104CF000CDFF01220B49FFF7C9FF00220A4910002E
:104D0000FEF77AFA10BDC046F263FF1FD363FF1FA0
:104D10001BBD0011D563FF1F6709FF1FDB63FF1F6A
:104D20006609FF1F6509FF1FAEDE000070B5124C5B
:104D3000132220001149FEF725FB114D002817DD35
:104D4000AB78002B14D0431C2B7009236B7000230D
:104D500000190370287829000130C0B206F058FF0E
:104D6000297822000139C9B2002005F0DBFD70BDB1
:104D7000FFF7A6FFEEE7C046D563FF1FAEDE0000DB
:104D8000D363FF1F10B5114B1A781870002A0ED08C
:104D900000280BD10E4B1A78062A07D85423D3408B
:104DA000DB0703D50B4B187802F00EFA10BD002874
:104DB000FCD0074B1B78012B02D0033B022BF5D80C
:104DC000044B0121187806F043FEEFE7F663FF1F5E
:104DD0001D64FF1F1E64FF1F70B5514E514A52499A
:104DE0003070082005F02AFC0121022005F030FB7C
:104DF000022005F011FC0121002005F029FB002014
:104E000005F00AFC00F0BAFEFEF7FAF806F070FDB5
:104E1000032246494648FFF739FF2D2403000422A8
:104E20001C7044490130FFF731FF30230470424DBC
:104E3000424C437083702E3B062220004049EB8792
:104E4000FEF7A0FA062813D0200006F0B1FC0228D5
:104E500009D00321200006F01BFD8D23E3706E3B7B
:104E6000237119336371062220003549FEF7C4F916
:104E7000344B1B68FC335C64FFF758FF0020FFF7DE
:104E800081FF314C314A0121314B1278207802F0F8
:104E90005DF9304A304B12780021207802F056F943
:104EA00001222E4B1A702E4BDB78552B31D12D4B16
:104EB0003B325A722C4B2D4AAB81EA812B826A829B
:104EC0002021307806F044FE0120404205F076FDB6
:104ED0000120404205F012FEFFF714F9FEF7D6FE5E
:104EE00000F0A4FC01204042FEF79EFF012006F0E6
:104EF0001FFCF02001F0E6FA0121307806F0A8FD51
:104F0000307802F0BDFA1A4806F052FEFEF7D2FDE4
:104F100070BD6422174B5B7953431A000A32CBE70A
:104F2000F461FF1F654B0011614C00115843FF1FD6
:104F30009061FF1FB061FF1FE242FF1F6509FF1F65
:104F4000ADAC00004064FF1F1E64FF1F3842FF1F0E
:104F50001942FF1FF263FF1FD363FF1FC463FF1FCC
:104F6000D461FF1FC861FF1FC4090000CE09000003
:104F7000F661FF1FD861FF1FF8B50A0020230D005E
:104F80001A40194257D0574B1B78002B50D0FFF7CF
:104F9000E5FA554B554C564E99686268737A8A1AF1
:104FA000DB039A4202D36160FEF784FD327A217AF4
:104FB000531EDBB2994205D1FFF75CF9002000F0E7
:104FC000A5FD0FE09142F9D300232372FFF77CF98E
:104FD000012000F09BFD474F3800FEF773FE3900BB
:104FE00006F036FE637A002B1FD0013BDBB2637202
:104FF000002B1AD1404BDB78552B01D106F0F0FD88
:10500000E37A002B0CD000233C4A3A4FE37213881A
:10501000380001331380FEF755FE390006F018FE04
:10502000642370795843FFF79FFD237A013323727D
:1050300020206840F8BD0BB2002B0ADA304B1878FC
:1050400006F08EFB002801D006F0E2FC8020000272
:10505000EFE70224214206D0244B01201A72FFF709
:1050600091FE2000E5E70B071ED5FFF777FA1E4BF0
:105070001E491F4C98684A68637A821ADB039A4279
:1050800002D34860FEF716FDFFF71EF9FFF7F2F8AE
:10509000012000F03BFD00F0E3FB2368DB0701D5B6
:1050A000FEF7BAFF0820C4E71024214206D00D4BBA
:1050B0001B78002BD5D1FEF7FDFDD2E7012421425C
:1050C00007D0104800F06CF806F0B2FA00F004FDCA
:1050D000C7E70424080020402142ABD0FEF7C0FE01
:1050E000BFE7C046F663FF1FE461FF1FC861FF1FF3
:1050F000D861FF1F1942FF1FD461FF1FBC61FF1F52
:10510000F461FF1FFC41FF1FF0B51B4B1B4F1B88B9
:105110003A8804001A4E1B4D85B09A420DD8328849
:105120009A420AD3184B1A882B889A4205D1174AFB
:10513000174B12881B889A421BD0052001F018FAE1
:105140003B8802AA13803388019053802B88114D2D
:1051500093800F4B02A91B88D3800F4B2A781888A5
:1051600002F034FF0D4B08212878019A1C7006F0DC
:105170002FFD05B0F0BDC046C263FF1F0E42FF1FEA
:105180000C42FF1F0A42FF1FC063FF1FBE63FF1FC9
:105190000842FF1F1E64FF1F1042FF1FBC63FF1F5A
:1051A00013B50C4B1C78002C11D1002801D00A4BF0
:1051B00018600A4A0A4B11780A4A10780A4A019282
:1051C0000A4A0092002205F0A5FA200016BD11241B
:1051D000FBE7C0461D64FF1FB863FF1F1C64FF1F71
:1051E0000C64FF1F1E64FF1FF863FF1FFC63FF1F9B
:1051F00010B5064B12201B78052B06D1044B132249
:105200001988044B187801F08FFB10BD1D64FF1F37
:105210001042FF1F1E64FF1F10B500240122114B16
:1052200052421870104B1C70104B1A8002F028F973
:1052300004220F4B21001A700E480C3206F0E8FAD7
:10524000102221000C4806F0E3FA07220B4B1C60E9
:105250000B4B1C700B4B1C700B4B1A700B4B1C70C8
:1052600010BDC0461E64FF1F1D64FF1F1042FF1FBC
:105270001C64FF1F0C64FF1FFC63FF1FF863FF1F0C
:10528000D263FF1FD163FF1F1242FF1FD063FF1FB6
:10529000F8B5174C0600257806A814240078052DCB
:1052A00023D1B41F134FA5B21824BD421DD88D1FA2
:1052B000ADB2BD4219D8FA256D00AA4215D21D0023
:1052C0000D4F0A3DADB2BD420FD80C4C26800C4CA0
:1052D00021800C4900240A800B4A1380FFF714FF39
:1052E0000A4B0421187806F02BFC2000F8BDC046BC
:1052F0001D64FF1F790C0000750C00000E42FF1F9B
:105300000C42FF1F0A42FF1F0842FF1F1E64FF1FBF
:10531000F0B50BB20D0089B0002B00DB70E1A44E9C
:10532000307806F01DFA041E50D00378A22B00D16D
:1053300022E1D02B1AD0912B45D143780E2B42D1AC
:105340009C4B82889A423ED19B4A83681278052AF8
:1053500039D1032018567F2835D0984B1B68002B75
:1053600031D05B68002B2ED098472CE0807807283E
:1053700029D806F055FB0428183F3F74A8D8637855
:10538000002B0CD101218C4B19708D4B1A78002AFF
:105390005BD08C4B307801F0D9FE002855D0072225
:1053A000854B1A7051E061780029F8D1E378002B21
:1053B00011D0854A854B1278307801F0C7FE6070B5
:1053C0006378002BEBD1200006F022FB8020000246
:1053D000684009B0F0BD784B1B78022BF3D0012157
:1053E000307806F0CDF90028EAD10121307806F0B6
:1053F0002FFBE5E76378002BD1D16F4F032807D14E
:105400003B78052B02D101333B701EE00223FBE702
:105410006F4B1A886F4B0293002A0BD01B78002B1E
:1054200003D00121307806F0D3FB3B78062B04D162
:10543000013BE9E7029B1A70F7E7042B41D10121F8
:10544000029B3078197006F003FB5C4B1B68002B45
:10545000B9D01B68002BB6D0574A107884E7637820
:10546000554F002B27D10622211D5B4806F040FB3B
:1054700062895A4B5A491A80A2895A4B1A80E38989
:105480000B800521397058490A80584A1380228AB6
:10549000574B1A80574B1B78012B09D11F2001F065
:1054A00067F8FA22920042430421307806F090FB1C
:1054B0000022484B75E7312B00D070E70022454BA6
:1054C0001A700323A0E706220021434806F0A0F942
:1054D0000023454A04211380444A30781380444A0B
:1054E000138006F02DFB0821307806F029FBA37904
:1054F000083B5A425341304A03331370304B1B78F8
:10550000002B06D0334B30781A78002A06D001F0F1
:105510005BFE0122314B52421A8096E7012119703D
:1055200006F096FAF5E70821307806F009FB637873
:10553000002B00D047E72C4B2D4F0293E388029AB3
:1055400004211380294B307803932389039A138015
:1055500063893B8006F014F9002800D033E7264B1E
:105560001B68002B00D12EE7039902983A8809881E
:1055700000881B68984726E74379132B00D022E761
:105580000389012B0AD11D4B1B78022B06D1082160
:10559000307806F0D5FAFFF72BFE14E7052000F06F
:1055A000E7FF08210200307806F012FB0BE7C04647
:1055B0001E64FF1F051400001D64FF1FB863FF1F5A
:1055C0003842FF1F1942FF1FF263FF1FD363FF1F03
:1055D000F463FF1FF663FF1FC563FF1F1042FF1F29
:1055E000CC63FF1FCE63FF1FC263FF1FC063FF1F9B
:1055F000BE63FF1FC463FF1FB463FF1FBC63FF1FB5
:105600008020C001014200D0E2E6CB0731D5324B09
:105610001B78002B1DD0314E05AC3378052B1AD1E9
:10562000023B23702E4B21001B7823722D4B1B78DD
:1056300063722D4B187801F02DFD002809D007204A
:105640002A4B30701B68002B03D01B68002B00D046
:1056500098470120BCE60E20254B06221B782549E1
:105660002370254B1B78637002ABC01806F040FA1C
:10567000D8E7022308001840194209D0174B1B78BD
:10568000052B03D11D4B188806F01AF902209FE65E
:105690000424214203D0FFF737FD200098E60823B9
:1056A00008001840194200D193E6154B1C78012CD4
:1056B00003D0022C0DD008208AE6124B124A13495F
:1056C00013481B881288098800880094FFF7E0FDC2
:1056D000F1E7FFF78DFDEEE7F663FF1F1D64FF1F87
:1056E0001242FF1FD063FF1F1E64FF1FB863FF1F1E
:1056F000D263FF1F1342FF1FD163FF1F1042FF1F22
:10570000BC63FF1F0842FF1F0A42FF1F0C42FF1F1E
:105710000E42FF1F10B502A804880B20002C10D1E8
:10572000496808784978090201430C48814209D147
:10573000022119800A4B59881170DB7800205BB276
:10574000537010BD074C0A20A142FAD102211980E2
:10575000034B998811705B79F0E7C0466E2A000010
:10576000BC61FF1F6F2A0000F7B5150008AA168854
:105770004A680F4F14785278120222430A24BA4220
:1057800014D10122DBB2019200962A0005F0C8FE76
:10579000041E0BD1074B1B68002B07D068782A78B2
:1057A0000002104342425041013098472000FEBDA4
:1057B000022900003064FF1F30B501250379040081
:1057C000BFB02B4225D01449408805F015FA284275
:1057D0000CD0124B01A95B8D00220B8002234B8061
:1057E0000F4B5B888B80608802F0E6FA0D49608879
:1057F00005F002FAC0070CD50B4B01A91B8800224B
:105800000B8002234B80064B9B888B80608802F0C4
:10581000D3FA3FB030BDC0462864FF1F3C42FF1F93
:10582000BC61FF1F2064FF1F9642FF1F10B5074C8D
:105830000749200005F096F92000064905F092F985
:105840000721054A054805F04FF910BDFFFF00008C
:105850002864FF1F2064FF1F8CBD00113C42FF1F06
:1058600010B5024803F02AF910BDC046B95700111F
:1058700070B540253F2608210B4BC207D2172A409E
:10588000DD789C7835408C432A439C70DA7082071F
:1058900001D521439970400704D58022D97852421E
:1058A0000A43DA7070BDC046B442FF1F13210A4B91
:1058B000DA788A43123901400A43DA700222104230
:1058C00002D0D9780A43DA70400703D51022D9787C
:1058D0000A43DA707047C046B442FF1F10B5054B4B
:1058E000082419790A00A243002801D022000A43A3
:1058F0001A7110BDB442FF1F10B5054B2024D97892
:105900000A00A243002801D022000A43DA7010BD29
:10591000B442FF1F0821F8B5324D334BAE78040076
:105920000E40AE70984204DD67232B70273B6B70EE
:10593000F8BD2E4B984203DAE0232B701A3BF6E7B2
:1059400000232B706B7083B21A0029485F3292B229
:10595000284F82422CD9002C03DA5B421CB204236C
:105960002B70053420B20A2105F01AFF04B2FA2385
:105970009B009C4232DB08232A7813432B7064215E
:10598000200005F00DFF0A2100B205F079FE09B2F2
:105990002A787B5C13432B700A21200005F000FF5E
:1059A0000A2100B205F06CFE09B27B5C6A780AE05D
:1059B0006970002CDBDA5B421CB204232B70F522E9
:1059C0006B78092CE8DC13436B700A21200005F08A
:1059D00057FE09B27B5C1E43AE70A9E7632CCEDC98
:1059E000EDE7C046B442FF1F1B4E00001DFCFFFF49
:1059F0002A080000B7BD00110823F7B5194FCD00E4
:105A00003E7904001E403E71EDB2632806DD5F332F
:105A100033433B7140231D437D71F7BD03000933C0
:105A200005DA20235B4233433B71C623F3E70E4B79
:105A3000019300280BDA0423444224B23B710A216B
:105A4000200005F01DFE019B09B25B5CE3E709281D
:105A5000F5DD0A2105F0A4FE019B00B21B5C1E438C
:105A60003E71ECE7B442FF1FB7BD0011F8B50A4F15
:105A700005003B780E00002B0CD0084C2000FEF7F0
:105A800037FC33002A0020003978FEF725FD20007E
:105A9000FEF76CFCF8BDC0463464FF1FBC42FF1F1C
:105AA00070B50A4E0A4D06223100280005F0C0FFED
:105AB000002809D0074C31000622280006F018F80B
:105AC00007212000FFF7D2FF70BDC046B442FF1F80
:105AD000AE42FF1FAD42FF1FE622202110B50A4B48
:105AE0001A70203A5A701C329A70DA780A40DA70CA
:105AF000082219791140033A0A431A7127225A7170
:105B0000FFF7CEFF10BDC046B442FF1F70B5184B63
:105B10005C78002C2BD1002829D0164D0A210223B5
:105B2000E85E05F03DFE00B2FFF7F4FE0423E85EF8
:105B3000642105F035FE012100B2FFF75DFF13225D
:105B400020002B7A9A426041C0B2FFF7D5FE0320B5
:105B5000FFF78EFE2000FFF7A9FE074B18780538E7
:105B600043425841C0B2FFF7B9FEFFF799FF70BD3D
:105B7000D461FF1FBC61FF1F1D64FF1F70B50025AE
:105B80000A4C2000A571FEF7B3FB11233E21200033
:105B9000074AFEF7A1FCA84200D13E35054B200084
:105BA0001D700123A371FEF7E1FB70BDBC42FF1F16
:105BB000A6BD00113464FF1F0200F0B501270A489A
:105BC0000A4E51188B1A002B00DCF0BD0824157802
:105BD0004308684038404000805B013C58406D08F5
:105BE000002CF5D10132EDE7FFFF0000C8BD001128
:105BF000F0B500250F269D4200DBF0BD4C5D070986
:105C000044403440A400A05801357840F3E7000038
:105C1000F0B589B06A460D000B000F271100103552
:105C20001C780133260024093E401670547002325D
:105C3000AB42F5D12023024AFFF7DAFF09B0F0BDED
:105C4000CCBD0011F0B54E780B7889B036020C004F
:105C5000170001901E43012A61D9954B9E4200D83E
:105C600077E001339E421CD1062A17D1CA788B787F
:105C700012021A430B791B0413434A7912061A4382
:105C80008C4B5A6100221A705A808B4A5A608B4A98
:105C90009A608B4ADA60002009B0F0BD8822520574
:105CA000EEE7884B9E423CD182498B78002B00D096
:105CB000F6E00C2A31D10F22A3789343E278120246
:105CC00013432279120413436279120613434B6083
:105CD000E279A07912020243207A00041043627A2A
:105CE00012060243CA60E27AA07A120202437648A0
:105CF0004A81834208D804236E49142201980B700C
:105D000005F0F6FE1420C7E71201D21889235B05BF
:105D10009A42F0D801238B70BDE7022AFAD00523FE
:105D2000EAE76A4A01239642E6D1FFF761FA052FB6
:105D30000CD9E378A2781B021343227912041A4388
:105D400063791B061343624A0393136005F048FF0F
:105D5000A1E7584D2B78002B9DD1AB78002B00D1BB
:105D6000A0E02B8901339BB20093B34200D091E0B5
:105D7000132AD4D9CF7C8B7C3F02122120001F43F1
:105D8000FFF71AFF874200D08EE0002E3DD1E37866
:105D9000A2781B0213432279E96812041A4363793B
:105DA0001B06134303930A228B4212D1FF23A370D5
:105DB000E370237163716B89002B09D1E37B227C33
:105DC0001B0212041343A27B13431B0901336B8193
:105DD00000226B89002B8ED0002A67D168683701BA
:105DE0003818000B6B6900030390984205D968616D
:105DF00005F026FDEB780133EB7068681022A11CDA
:105E0000381805F0F5FE2E8145E76F89009A7B1E54
:105E10009BB293423AD1E278A37812021A432379D3
:105E200005A81B04134362796C6812061A43EB68D9
:105E300000920392211D0C22049305F059FE0120CB
:105E4000260004A940421036FFF7E2FE013F012F71
:105E500017D1009A0B232861824200D04CE704221C
:105E60001C49200005F0C4FE042203A9686805F05F
:105E7000C7FEE968039AFF23914200D13CE7F73B54
:105E80003AE73100FFF7C4FE1036DFE70923B742D7
:105E9000A4D831E7009BB34200D9FCE607232BE7E7
:105EA000022329E7032327E7062325E70A2323E71D
:105EB000FFFE0000C442FF1F00000111FFFF0000B1
:105EC0005048593601FF0000FFFF001102FF00009B
:105ED00034F00040D042FF1F10B5034C0B000122EC
:105EE000210000F06BFA10BD996000110B8870B5AD
:105EF00006000D000224162B11D92B00032209499C
:105F000000F05CFA041E0AD1074B2A881B88191C72
:105F1000934200D9111C300089B200F0EFFA200042
:105F200070BDC046C56000115A64FF1F10B54A78A5
:105F30000400013A0B000220012A07D80A78002A3F
:105F400004D005222000024900F038FA10BDC046F6
:105F5000F36000110A7810B50B0004000220002A3B
:105F600004D007222000024900F028FA10BDC046E4
:105F70009F6100110A7810B50B0004000220002A6E
:105F800004D009222000024900F018FA10BDC046D2
:105F90000562001110B5034C0B000B22210000F02C
:105FA0000DFA10BD3562001110B5034C0B000D2227
:105FB000210000F003FA10BDA762001110B5034CD8
:105FC0000B000F22210000F0F9F910BD0163001150
:105FD0000A7810B50B0004000220002A04D0112218
:105FE0002000024900F0EAF910BDC046116300111B
:105FF000002310B51322190000F0E0F910BD0000D5
:1060000010B5034C0B001722210000F0D7F910BD8A
:1060100063630011002310B51922190000F0CEF9B6
:1060200010BD000010B5034C0B001B22210000F036
:10603000C5F910BD9D630011F7B584890D000600F8
:106040000121002C22D000238268D3561778002B20
:106050001EDA0C2C1AD90C3CA4B2131940880093F8
:10606000230002F086FE431E984101307B06DB0FC1
:106070006B703F23013C1F40A4B22870AF70AC800E
:10608000002C07D0B3680133AB6000210800FEBDCF
:106090000020EBE7AC60F8E70B7803704B884370A7
:1060A0004B881B0A83700B79C3700420704704204F
:1060B000022B06D10020537811781B02009A0B4363
:1060C000138070470B8803700B881B0A43700220F3
:1060D00070470420009983420AD1537810781B023C
:1060E00003430B80D37890781B02034300204B803E
:1060F0007047F8B50D004B7801240021461C037051
:106100002B788B4201D82000F8BD6B78B01C4F1C57
:10611000012B10D1890069184B88022233704B88FB
:10612000B9001B0A7370691805F0BAFC0436043410
:10613000A4B2F9B2E4E7122359436B185A88043128
:1061400032705B8810221B0A7370691805F0A8FC76
:1061500012361234ECE770B5049D14001E00052BB6
:1061600001D8042070BD637812781B0213432B8082
:10617000E378A2781B02134302226B802A71211D4F
:10618000681D063E05F08CFCB2B22A81E92AE8D8E7
:106190002800A11D0A3005F083FC0020E2E700235F
:1061A00010B50A789A4201D8900010BD9A008A185A
:1061B0005488013304705488DBB2240A44709488F4
:1061C00084709288120AC2700430EAE710B5110098
:1061D000029C062B04D004201022142B01D010BDE9
:1061E000022222714B7808781B0203432380CB786C
:1061F00088781B02034363800431601D05F050FC66
:106200000020ECE710B50C788B7804315C43E4B2E5
:1062100003702200013005F043FC601C10BD042017
:10622000022B06D10020537811781B02009A0B43F1
:106230001380704710B50C000A88023105F030FC5D
:10624000208810BD70B504000D0004981100012BCA
:1062500001D8042070BD16785278120232430280B1
:106260000200F13255701470E125002C00D10C357C
:10627000023B9AB24280AA42EBD80231043005F0C8
:106280000FFC0020E6E70420009983420AD15378EE
:1062900010781B0203430B80D37890781B020343D2
:1062A00000204B80704710B50C000A88023105F0C1
:1062B000F7FB208810BD000070B501211E000420EE
:1062C000049C0E400B4218D1CB40DDB28D4214D954
:1062D0000A49DBB2098899420FD32300EE331D70BF
:1062E0003300580011184978165C09023143013314
:1062F0002152D9B28D42F4D8002070BDDC42FF1F7C
:1063000010B50C000A88023105F0CAFB208810BDC8
:1063100010B50C788B7804315C43E4B20370220032
:10632000013005F0BDFB601C10BD10B511000298D6
:10633000032B01D8042010BD14785278043B1202BC
:1063400022430280CA788C781202224342809AB299
:106350008280EB2AEED80431063005F0A1FB002044
:10636000E9E710B50C000B8803700B881B0A43701B
:106370004B8883704B881B0AC3708A8804300631AF
:1063800005F08EFBA088043080B210BD0420012BE4
:1063900003D100201378009A1370704710B50C00D9
:1063A0000B8803700B881B0A43704A880230043143
:1063B00005F076FB6088023080B210BDF0B589B080
:1063C00003931E4B029242000700D05A019102F043
:1063D00020F81325061E2DD0029B01240370019B7B
:1063E000002B04D0001903999847001984B26B461A
:1063F0001B7A5BB2002B0FDA1021380002F01CFB75
:106400001925002813D130003219E1B202F066FCE0
:10641000051E0CD10C34A4B2042304AA380005A92B
:1064200093800696948101F0AFFD051E02D03000E6
:1064300005F0AEFB280009B0F0BDC0465864FF1F50
:1064400070B505000C0000280CD00020814209D056
:1064500010222000044905F023FB01202B78237330
:106460006B78637370BDC0460CBE0011F0B50600BA
:106470000D0017001C0085B002291BD00020102938
:1064800007D1022B07D0102B03D115E00020102CD0
:1064900008D005B0F0BD69463800FFF7D1FF2A00EB
:1064A00069460BE069463000FFF7CAFF22006946E3
:1064B000380004E0022BE9D12A003900300005F051
:1064C0005FFBE6E7031CF02800D9F023032008490E
:1064D0009AB2013A0B80D317034006499B189B10D0
:1064E0000B80D30F04499B185B100B807047C0468C
:1064F000E042FF1FDE42FF1FDC42FF1F034B1B88F1
:106500008B4202D3024B4000C1527047E042FF1F52
:106510005864FF1F014B4000185A70475864FF1F12
:106520001722014B1A8070475864FF1F70B5050091
:106530000E2005F01DFA041E13D0D0230370002393
:106540000622837007494570033005F0A9FA064B0F
:106550002100DA8A62811B7E2373044B187805F0D0
:10656000C7F870BD7464FF1F6464FF1F3043FF1FD2
:10657000262803D8024B4000C05A70470148FCE768
:10658000E242FF1FFFFF000070B506000C00094D3E
:106590001C220021280005F03BF9074B1E70074B19
:1065A0001C7005F02DFA0123002801D000231220D1
:1065B0002B7070BD6464FF1F3043FF1F8564FF1F95
:1065C00070B505000D4C0800E260A16010220021AA
:1065D000656005F03DF8012803D11021A06802F0A4
:1065E00058FD10220021280005F032F8012803D1BF
:1065F0001021606802F04DFD70BDC0466464FF1F4D
:1066000070B5041E05D1002903D006220D4805F0FF
:1066100047FA0D4B1D78012D11D1002C05D1022216
:106620001A7005F05DFA280070BD00221A70074B41
:106630001B78FF2BF7D02000FFF778FFF3E700254A
:10664000F1E7C0467464FF1F6464FF1F3043FF1FFF
:10665000030010B5002801D1002010BD00780B4ABE
:10666000002803D15988D1821B7913761378022B25
:10667000F2D10023984200D103331370044B1B78EE
:10668000FF2B01D0FFF752FF0120E6E76464FF1FF4
:106690003043FF1F002911D000280CD04B7901286E
:1066A00003D140225242134303E03F221340032808
:1066B00002D001204B7170474022F4E70800FAE74E
:1066C00070B5094D0100287800280BD0074C062230
:1066D000200005F0E5F921002878FFF7DBFF200016
:1066E00005F00EF870BDC0468464FF1F5E64FF1F96
:1066F00000290AD0012808D13F224B799343C02BAF
:1067000003D0403B5A425341981C704770B5174D17
:1067100006002B78FF2B15D00A2005F029F9041E5E
:1067200010D0D0230370C83B8370114B11491B78E4
:106730004670C3700622043005F0B2F921002878B3
:1067400004F0D6FF0C4B1B78012B0DD10B4B1B68B3
:10675000002B03D09B68002B00D09847084B0421E6
:106760001878084A05F044F870BDC0463043FF1F52
:106770008464FF1F5E64FF1F8064FF1FAC64FF1F03
:10678000B064FF1F60EA0000014B98687047C04684
:106790006464FF1F014BDB68186870476464FF1F67
:1067A000074B10B5DA68136801331360054B18788E
:1067B000FF2803D08021C90105F04AF910BDC04669
:1067C0006464FF1F3043FF1FF7B50E0002F0C8F8E6
:1067D000051E1CD00E4B06621F78002F00D10778D3
:1067E000AB791020019305F0C3F8041E0FD0D0231D
:1067F0000380C73B8370019BE91DC37006220430F0
:1068000005F04EF921003800E66004F071FFF7BD95
:106810002E43FF1F014B18787047C0468464FF1F4A
:10682000054B002805D1054B1A78054B002A00D1ED
:10683000014B18007047C0467464FF1F8464FF1F3B
:106840005E64FF1F014B58687047C0466464FF1FB9
:10685000024B1868431E9841C0B270478864FF1FFE
:10686000421E03000120152A03D9FF3B5A4253411F
:10687000D8B27047F0B51C0000230E0085B003901D
:1068800002920B70029A934201D3002019E0E55C5A
:106890005A1CD2B2002DF8D0029851198142F4DC72
:1068A0000233DFB2A35C18000193FFF7D9FF002881
:1068B00007D0013D019A0399EBB233708A4202D1AD
:1068C000E01905B0F0BDDB19DBB2DBE710B50C0059
:1068D00002F09EF803001220002B03D021005888FC
:1068E00004F02EFF10BD000070B50E4D84006359FA
:1068F000002B15D0186A002801D004F009FF2B598D
:10690000586A002801D004F003FF2B59986A002828
:1069100001D004F0FDFE285904F0FAFE00232B51AB
:1069200070BDC0469464FF1F1C4B70B504000E0080
:10693000150099420AD11A4B1B68002B01D1122075
:1069400070BD1B68002BFAD09847F9E7154B9942A8
:1069500015D1134B1B68002B0AD01B68002B07D0E6
:106960009847002804D1104B1C70104B1D70E7E7AE
:1069700029002000FFF7AAFF0028E1D1F3E7080073
:1069800001F0EEFF0028DAD003780320A342D7D12C
:106990002900300004F0D4FED2E7C046FEFF00001C
:1069A0009064FF1FFFFF00008D64FF1F8C64FF1FBA
:1069B000F7B50400808801F0D3FF0025A84203D07A
:1069C0000578A08802F008F81C4E3378002B1FD001
:1069D000AB421DD11A4B28001978FFF777FF00282A
:1069E00018D000233370A3790820A778A6880193D4
:1069F00004F0BEFF011E0DD0D0230370CA3B83708C
:106A0000019B477086808371280004F071FE01E0CD
:106A1000002DE8D1A0880B4B8200D358002B01D069
:106A2000FFF762FF1721A088FFF768FDA08801F03B
:106A300027FDA08801F0FEFDF7BDC0468D64FF1F55
:106A40008C64FF1F9464FF1FF0B587B01D000CAB72
:106A50001B88070001930DAB1B88142002930EAB1B
:106A60001B88160003930FAB1B880091049310AB97
:106A70001B88059304F07CFF041E1AD0D0230370FA
:106A8000CB3B47708370C670062229000430002D6E
:106A900011D005F005F8019B21006381029B00984D
:106AA000A381039BE381049B2382059BA37404F0D1
:106AB0001FFE07B0F0BD04F0ABFEECE7F7B50093A6
:106AC00008AB1B8807000C200D001600019304F092
:106AD0004FFF041E13D0280001F042FF00280FD002
:106AE0000078D0232370C93BA370009B2100238131
:106AF000019B6770A580E680638104F0F9FDF7BD16
:106B0000014B1878EDE7C0463043FF1F13B5040072
:106B100064890389C2888188C0780094FFF7CEFF1A
:106B200013BD000010B5044C2068002803D004F009
:106B3000EFFD0023236010BD9864FF1FA122F0B574
:106B4000818892004A43384B384F1B6804009B18D9
:106B50009D2292009B18827989B01A603B68002BB5
:106B60005FD01D78324B1B68002B04D05B68002B74
:106B700001D000209847260008363100E079FFF761
:106B8000B7FD237DE0710200E0780493638A290059
:106B90000393238A0293E3890193A388009333002C
:106BA000FFF752FFE378002B0BD1E289A379A1888C
:106BB00002920196E27928000092012201F0DAFEA9
:106BC000E0703B68002B20D0FFF7ACFF194D287810
:106BD00000281AD0184B1978FFF778FE002814D037
:106BE0002B78E67808200793A78804F0C1FE011EE1
:106BF00009D0D0230370CA3B4670837087808671AA
:106C0000079804F075FD00232B701721A088FFF76B
:106C100075FCA08801F034FCA08801F00BFD09B0E0
:106C2000F0BD064B9DE7C0463409FF1F9864FF1F67
:106C3000AC64FF1F8D64FF1F8C64FF1F3043FF1F78
:106C4000F8B5070008000E0001F08AFE041E18D0F7
:106C50002620FFF78DFC051E00D12578062004F0C4
:106C600087FE041E0DD00021062204F0D1FDD023A2
:106C70002370C23B21006770A370A680E8B204F0C5
:106C800037FDF8BDF0B585B001930AAB1B7807005E
:106C900002930BAB1B7808000D000092039301F0E8
:106CA0005FFE061E22D0102004F062FE041E1DD0DE
:106CB0001022002104F0ACFD2620FFF759FC00282B
:106CC00000D13078D0232370C13BA370009B2100FA
:106CD0002372019B67706372029BA580A372039B62
:106CE000C0B2E3720C9BE36004F002FD05B0F0BD9E
:106CF000F7B50D00019001F033FE071E20D00E20E5
:106D000004F036FE041E1BD02620FFF731FC061EC1
:106D100000D13E78D0232380C53B0622A370F91D05
:106D2000E01C04F0BDFE019B2A0063810123DD40CD
:106D30001A401D40210022736573F0B204F0D8FCA4
:106D4000F7BD0000F0B585B0029010000D001700EF
:106D50000A9E039301F004FE041E31D0029B002B17
:106D60002ED1039B02795B0724D5122313430422FF
:106D7000002E08D10B99002905D10C99002902D1C8
:106D80000D9900291AD01A430D9B2271002B00D0B7
:106D9000C9E0002E00D1CFE0002D00D0CCE0606A29
:106DA000002801D004F0B4FC1C21300004F020FEC7
:106DB000606205E002239A430E33D7E793432371C1
:106DC000654BBA00D458002C00D1AAE0002E10D098
:106DD000236A002B03D11C2004F0C2FD20625E4B0D
:106DE000BA00D358186A002803D01C22310004F0DE
:106DF00057FE0C9B002B12D0574CBB001D596B6AE1
:106E0000002B03D1162004F0ABFD6862BB00E358F1
:106E1000586A002803D016220C9904F041FE0D9BFD
:106E2000002B11D04C4DBC006659B36A002B03D126
:106E3000142004F095FDB0622B59986A002803D005
:106E400014220D9904F02CFE380001F089FD051E76
:106E500067D0414BBA00D358002B62D01A6A342055
:106E6000002A00D11C389A6A002A01D0143080B25E
:106E70000B9A002A01D01C3080B25B6A002B01D033
:106E8000163080B204F074FD041E4AD0182200218E
:106E900004F0BEFC2620FFF76BFB0190002801D117
:106EA0002B780193D0232370029B200063700A2368
:106EB000294EA370039BBD00A371AB59A780196A2B
:106EC0001830002905D01C22A06004F0E9FD200044
:106ED00034307359996A002907D0030014221433FF
:106EE000E060029304F0DCFD02980B9B002B08D0BD
:106EF00003001C221C330B992061029304F0D0FD87
:106F000002987359596A002903D01622606104F06F
:106F1000C7FD6B462100187904F0EAFB3800FFF743
:106F2000E3FC05B0F0BD10220D9B0D991B69A01864
:106F3000236204F0B5FD2CE70B9B002B00D13FE74B
:106F4000012D00D03CE7606A002801D004F0E0FB8E
:106F50001C210B982AE7C0469464FF1F10B5044C0F
:106F60002068002803D004F0D3FB0023236010BD69
:106F70008864FF1F0B4B07B51A68002A01D1002057
:106F80000EBD6946531C012012780731FFF772FCD1
:106F90000028F4D002780123100018401A42EED0E5
:106FA000EEE7C046A464FF1FF0B51F4F01203B6809
:106FB00087B0002B25D09B78059300F0B3FB002809
:106FC00021D00A20FFF7D4FA04000B20FFF7D0FAF3
:106FD000164B05001E78731E9E413B68F6B2191DC4
:106FE000D878FFF757FB3B682900DA7A043303921D
:106FF0009A7901930292009033002000059A04F0E0
:107000003FFD07B0F0BDFFF7B5FF002805D0062013
:10701000FFF7AEFA04000720D8E70820FFF7A8FA28
:1070200004000920D2E7C0468864FF1F8464FF1F64
:1070300070B50A4E040033780D00FF2B0DD00420EC
:1070400004F096FC011E08D0D0230370CE3B45709F
:107050008370C470307804F04BFB70BD4043FF1F59
:1070600070B5040006200D0004F082FC011E0AD059
:10707000D0230370CD3B8370054B44701B68858023
:10708000187804F035FB002C01D0FFF767FF70BDC6
:107090008864FF1FF8B5264F06003B680D001124D9
:1070A000002B05D10522234B1B78134202D1122459
:1070B0002000F8BD204A10241268002AF8D0127867
:1070C000002AF5D0DB0719D52B789A1E012A1AD889
:1070D0000C2004F045FC132438600028E8D000237D
:1070E0000A22437029000670023004F0D9FCFFF731
:1070F0005BFF041E0AD0FFF731FFD9E700F012FB57
:107100000028E1D1E4E7002BE2D0D0E70B4B1B785D
:10711000032BCDD11D20FFF72BFA094B1880002837
:10712000C6D0084B04211878074A04F061FBBFE77A
:107130008864FF1F8564FF1FA464FF1F8464FF1F12
:107140008264FF1FB064FF1F60EA0000F7B501937F
:10715000194B14001A78052306000F0012201A425A
:1071600021D0012920D1154B1D68002D1BD00220F4
:107170001F2C18D8002C02D0019B002B13D0104BD1
:107180001F221E706E1C0021300004F041FB01998B
:107190002200300004F084FC310020002C70002F0D
:1071A00006D004F075FCFEBD064B12201D68DCE71E
:1071B00004F02EFDF7E7C0468564FF1FA464FF1F9F
:1071C0004043FF1FA064FF1FF8B50F4E1224336821
:1071D000002B17D01B780F3C834213D100250B4F97
:1071E0000221387804F0ACFC094B042138781D806A
:1071F00004F0A6FC074B28001D8033685C7004F087
:1072000067FA04002000F8BD8864FF1FB064FF1F08
:107210009C64FF1F8264FF1F70B5012823D11B4CA3
:107220002388002B03D01A4A1578002D07D0194B5C
:107230001B68002B02D01878FFF7C6FF70BD3B2BF0
:1072400002D93C3B2380F9E7134E0221307804F049
:1072500077FCFA222388920002215A43307804F006
:10726000B7FC2580EAE70B4B1B68002BE6D00B4BE5
:107270001B785B07E2D5084B0221187804F060FC0C
:107280000022024B1A80FFF769FED7E79C64FF1FBC
:107290008064FF1F8864FF1FB064FF1F8564FF1FA9
:1072A000F8B51E4D2868002803D004F031FA0023F9
:1072B0002B601B4E3068002803D004F029FA00230D
:1072C0003360184F05243B7818002040234221D01A
:1072D000154800F02BFA3B78234213D0202004F00D
:1072E0003FFB2860002813D02022002104F090FAF0
:1072F000202004F035FB041E306005D02022002140
:1073000004F086FA002004E0286804F001FA2C60FA
:107310001320F8BD00F00AFAF4E7C046A464FF1F8A
:10732000A064FF1F8564FF1F3443FF1F10B50A4C84
:1073300023681A1E0ED0002808D10130587004F0BE
:10734000C7F9002805D02368002B02D00021FFF7E1
:1073500087FE0122100010BD8864FF1FF7B5274E7D
:10736000050033680191181E21D05C78244F012C50
:1073700030D1FFF7FFFD002825D02000FFF7F8F8F7
:107380000400412814D91F4B022118781E4A04F02A
:107390002FFA1E4B3C3C1C80022233685A703B780B
:1073A000002B14D128000199FFF75AFE0120FEBDE1
:1073B000FA2292004243002AEED0124B02211878A2
:1073C00004F006FCE8E7FFF7D3F80200F3E7002338
:1073D0003B70EBE73B78002BE8D1032004F0C8FAC0
:1073E000011E08D0D0230370CC3B457083703368F6
:1073F000187804F07DF9FFF7B1FDD7E78864FF1F27
:107400008064FF1FB064FF1F60EA00009C64FF1FE0
:1074100010B51749838802008B4220D011D8154936
:107420008B4217D0144900205B1899B2012907D864
:10743000926811785A425341D8B2FFF7F9FD012002
:1074400010BD0E4A00209B1807229BB29A42404171
:10745000C0B2F5E783681878FFF768FFF0E7836844
:1074600099785A78090218781143FFF777FFE7E710
:107470000A20000006200000F8DFFFFFAFDFFFFF5B
:10748000014B18707047C0464143FF1F10B5064CB2
:10749000207001F041FA207804F092F9052120785B
:1074A00000F062FD10BDC046B064FF1F0BB273B5A3
:1074B0000D00002B00DBC4E0884B187804F050F975
:1074C000041E0ED00378912B0FD0A22B00D1A1E087
:1074D000834B1878FF2852D0210004F009F90028C6
:1074E0004DD180200002684076BD43780F2B76D0C6
:1074F00013D8052B70D00E2BEAD18088794B984297
:107500002BD8794B98421BD8784B9842E0D1A3688E
:107510001878591CFFF774F838E03E2BD8D18378DF
:10752000032B74D06CD8012B6ED0022BD0D1704BB2
:107530001B68002B23D05B68002B20D098471EE0EF
:107540006C4BC0180C28C3D804F062F81DC2C215D9
:107550000BC20B0B0B3223C23C00674BC018072831
:10756000B6D8664B1B68002B09D01B68002B06D0D1
:10757000200098470AE0A3681878FFF7C7F82000B2
:1075800004F046FAADE7A068FFF762F800289FD044
:10759000F5E7A3681B78002BF1D0554B1B68002B37
:1075A000EDD01B68002BEAD0210055489847EDE745
:1075B0004F4B1B68002BE2D01B68002BDFD0210053
:1075C0005048F3E7504B1B68002BD8D05B68002B6A
:1075D000D5D021004348E9E7FFF7EAF9CFE78088F3
:1075E0004A4B984203D04A4B984200D070E7464B32
:1075F0001B68002BC3D05B68002BC0D02100D5E7EF
:10760000153B012BBBD963E7FFF798FAB7E7FFF704
:107610007DFAB4E73F4B1B78042B07D100236A4661
:1076200013800179408800F0C5FCA8E7364B1B6841
:10763000002BA4D05B68002BA1D0010036489847EE
:107640009DE7012421420AD0294B1B68002B04D05E
:107650005B68002B01D000209847012043E78B078F
:107660000AD5264B1B68002B04D05B68002B01D089
:1076700020009847022036E70421280008400D42E8
:1076800000D131E7254E3388002B21D0013B9BB23E
:107690003380002B1AD1FFF7DBF800280AD0204BEB
:1076A0001C70164B1B68002B04D05B68002B01D0AC
:1076B00020009847FFF7C6F8694601F001FD6846CB
:1076C000FEF7FEFF1D20FEF753FF308004200AE77F
:1076D000024B187804F034FAF8E7C046B064FF1F94
:1076E0004143FF1F0E200000012000000910000090
:1076F000A864FF1FFEDFFFFFAFDFFFFFAC64FF1FCB
:107700000C2000000B2000009064FF1F0D200000E3
:10771000132000008564FF1FFFFF00008264FF1F2D
:107720008064FF1F10B501F09BF910BD014B18607C
:107730007047C046AC64FF1F0B880020162B01D891
:1077400017230420014A13807047C0465A64FF1F64
:1077500000207047074A03001188814207D09188B2
:107760000020994202D1013080001018704700209B
:10777000FAE7C046B864FF1FF0B58F7806000D0029
:10778000C5B01E2F15D1FFF7E5FF051E03D100245C
:10779000200045B0F0BD00223B003100C0780092CF
:1077A00000F0B2FB0400A81C00F0D2FBFF23EB703A
:1077B000EEE7264B062403931B78FF2BE8D0182F07
:1077C000E6D87B08224A013BDB0002929A58944695
:1077D000002ADDD0029AD3185B68002BD8D0087835
:1077E000002802D14B78012B02D10624122FCFD1D1
:1077F00007AFAB88697800976446AA68A047041E63
:10780000C6D1AB78029A5B08013BDB00D318390084
:1078100030005B689847041E0BD1AB78042BB6D0C0
:10782000039A310010782200009700F06DFB0400ED
:10783000AEE76A78002AABD1AA7805A93B8808711F
:1078400030000A704B80FEF747FBA0E74443FF1F60
:107850001CBE00111D4B37B5050098420BD0002906
:107860000AD1FFF777FF002805D11948FFF772FF0B
:10787000002800D0058037BD01291AD1FFF76AFF23
:10788000041EF8D001235B420380A378FF2BF2D0C3
:10789000FE2B07D00023E0781422009329001E332A
:1078A00000F032FBA01C00F053FB01235B4263801D
:1078B000E1E70229DFD1013901F0BEF80028DAD171
:1078C0002800FFF747FF041EDFD1D4E7FEFF0000CA
:1078D000FFFF0000022210B5074B52421A800748F2
:1078E00001325A809A80DA8000F07EFA044801F072
:1078F00025F8002010BDC046B864FF1F797700113D
:10790000557800110388F7B50400002B02D1022539
:107910002800FEBD42680221137825485268FEF710
:10792000A5FD00282ED0234F01253A88002AEFD04C
:10793000802321885B0201259B1A9942E8DC0C20F8
:1079400004F00EF8061E31D03B8822889C460023A6
:107950001800019561469DB2491989B2AA421BD807
:10796000002801D062443A8000233000082208C079
:10797000210004F095F8104A1368002B13D100255C
:107980001660C5E76268022113780C485268FEF75A
:107990006DFD0028C7D1BAE760681D01401941811B
:1079A00001330198D6E71A001B68E6E71325AFE715
:1079B0008ABE00114243FF1FB464FF1F88BE00113E
:1079C000014B18707047C0464443FF1F14230A0040
:1079D00010B51A40194204D00122102101F048F8D4
:1079E00010BD4B06F9D4012088434000F8E710B5DC
:1079F00014008B0604D50122102101F039F810BDC6
:107A000008230A001A40194202D14BB2002B0FDAA8
:107A1000102101F02DF8002808D02300F2331B7844
:107A2000002BECD0F1342378012BE8D10020E6E7DD
:107A300003208907FAD4E2E7F0B51F00184B85B0A0
:107A40001C68019002910392002C27D1200005B000
:107A5000F0BDA5683301ED186B89019A934211D3EB
:107A6000029A93420ED8002F04D10A9B002B10D10A
:107A70002C00EBE73B002978039A6868FEF7F6FCD8
:107A80000028F2D10136B6B2A388B342E1D8246807
:107A9000DAE7A3680A9A5B891380E9E70026F3E72F
:107AA000B464FF1F37B50C000A884988012391424E
:107AB00017D3002A15D0651D23792A0002210A4810
:107AC000FEF7D4FC102300280BD02379618820888E
:107AD00000242A000094FFF7AFFF0A23A04200D041
:107AE000230018003EBDC0468ABE001113B50A002F
:107AF00008884988012388420BD8002809D000242F
:107B0000137905320094FFF797FF0A23A04200D0B3
:107B10002300180016BD13B50A0008884988012300
:107B200088420BD8002809D000241379053200942C
:107B3000FFF782FF0A23A04200D02300180016BDE1
:107B4000F0B58BB003904A8808880E00012382426A
:107B500055D3002853D00023012704AC2370002202
:107B6000718813000092FFF767FF051E3ED0207852
:107B7000002835D12B78022B18D167706A898300D1
:107B80000130E31880005A8069680222201803F04F
:107B900087FF23780133DBB22370042B19D93B0014
:107BA0006889013080B2002BD9D01FE002236370B6
:107BB000122358436A89231804305A8069681022B6
:107BC000201803F06DFF23780133DBB22370002B04
:107BD000E5D10C4A6B899B185A425341DBB2DFE76F
:107BE0006378012BE4D12B78022BC7D022780A23AB
:107BF000002A04D021000398FEF798F9002318000A
:107C00000BB0F0BD0100FFFF0F4BF0B5040018688A
:107C1000002816D083685D89A54207D88288AE18EF
:107C2000B44203DA12019A18934201D10068EFE7D7
:107C30001E005F891036A74204D1002900D00D80B4
:107C40001800F0BD3300EFE7B464FF1F70B5050006
:107C50000C0008880021FFF7D7FF03000120002B4C
:107C600004D022002800197AFFF7C1FE70BDF7B5D5
:107C70000C00002501902300EE331B78AB4201D8A5
:107C800000200AE06B00E65A00213000E718FFF7F9
:107C9000BBFF002802D126800130FEBD017A019889
:107CA000FFF794FE002802D03B882380F5E70135DA
:107CB000EDB2E0E710B5040008880021FFF7A4FF4B
:107CC00003000120002B03D02000197AFFF77EFE6D
:107CD00010BD0000054B1B68002B01D1180004E00B
:107CE0009A6852898242F6D198887047B464FF1F1F
:107CF000F0B50E27002687B0039302ABFF183E8035
:107D000005001F4B40891400984207D02B780130A2
:107D100000976A6880B2FFF78FFE060002212B7879
:107D200018486A68FEF7A2FB00280FD06C89200073
:107D3000FFF7D0FF002802D0013C0419A4B2039B36
:107D4000002B00D01C80300007B0F0BD02212B7842
:107D50000D486A68FEF78AFB0028E7D102212B78DC
:107D60000A486A68FEF782FB002807D0002EDED0A2
:107D70003B88A342DBD17489013CDFE76C89DEE7F5
:107D8000FFFF00008ABE001188BE001186BE0011F0
:107D900010B50C00FFF7DEFC03000220002B0AD018
:107DA000002C00D023609B781720FE2B03D00138D5
:107DB000FF2B00D1002010BD73B50D0001A90400F8
:107DC0001600FFF7E5FF172805D0002E04D1290083
:107DD0002000FEF727F976BD01221021200000F0D7
:107DE00047FE0028F3D0F6E7014B18607047C04605
:107DF000C464FF1F37B56B469D1D010004000222BD
:107E0000280003F075FE2B88B02B0ED12379122B9E
:107E100009D12300FA331B78012B06D10121608898
:107E200000F0E0F801E01B2BF8D037BD10B5054B92
:107E30000421187000F098F8FFF74CFDFEF770FB76
:107E400010BDC046C864FF1F0020F0B50BB20F0084
:107E500087B0834234DA274B187803F081FC051E83
:107E60002BD00378A02B25D103AE3100FEF7E4F828
:107E7000041E0BD1B378DB0724D51F4B06341B68D7
:107E8000002B03D03100688898470400A8680028B8
:107E900001D003F07DFE002C08D1184A039B13404B
:107EA000174A934206D0B3781B2B03D00121688870
:107EB00000F098F8280003F0ABFD80200002784025
:107EC00007B0F0BD0F4B1B68002B10D03100688845
:107ED0009847041EDAD07378002BD7D1B27801A965
:107EE0000A704B800C716888FDF7F6FFCEE7062418
:107EF000F1E7C046C864FF1FC064FF1F00FFFF001A
:107F000000011200C464FF1FF7B50190FC200D00B2
:107F100017001E0003F02CFD04001320002C12D0CB
:107F2000B02320002370089BF422677065802671BF
:107F30000830002B08D0190003F0B2FD2100019891
:107F400003F0D6FB0020FEBD089903F061FCF5E7C5
:107F500010B5041E06D00078FD2803D803F040FCBD
:107F6000FF23237010BD00000A1F93B210B5040058
:107F70000220032B05D882400020024BD1529B18CF
:107F80009C7010BDE864FF1F0B8870B5043B0400B3
:107F90000D000220032B0BD80121200000F04CFD26
:107FA00003001420002B03D02900200000F0DEFB8A
:107FB00070BD000007B51300034A00920A000121BA
:107FC00000F02CFC0EBDC046F181001107B50192F6
:107FD00003220092024B0A00122100F049FC0EBD60
:107FE0006F82001107B56B4601AA11800449D88041
:107FF00008780633012802D1190003F0A9FC07BD57
:10800000C964FF1F0C4B10B518700023FF210B4AE9
:108010001380138193819380094A538013705172A6
:1080200093819372D174D3821375517703F040FB1F
:1080300000F0FCF910BDC046F864FF1FE864FF1FA4
:10804000CA64FF1FF0B58DB06B46002003910C226F
:108050009B5E834200DBB0E05D4B187803F080FB51
:10806000051E00D1A4E00378902B00D09DE006AF60
:1080700001004688380000F013FA796804000029EE
:1080800000D19CE03B88052B6ED13B89032B1CD98A
:1080900005AC200000F0A2F86288172A61D839895F
:1080A000131D994231D17968237804310291D9079F
:1080B00038D5607800F08EF9071E06D000230371D2
:1080C0002378012B08D0132B23D0A868002800D1D7
:1080D00078E003F05DFD75E06288029909A800F080
:1080E000A6F80290380000F08BF909AA2378387AB4
:1080F0000192002231000092029A00F012F9380039
:1081000000F064F9029B002BDFD0300000F080F912
:10811000DBE70378032BD8D16288029909A800F025
:10812000D6F8DEE7122B13D1029909A800F0B5F8B2
:10813000021EEAD127498B88002BC6D0887909A96D
:108140002378019161780091310000F0EAF8BCE7F2
:10815000002302AA93833000617809AAFFF72AFF5F
:10816000B3E71D4B0993F6E7042B02D09A1F012AAF
:10817000ABD8184A043B9B00995A0029A5D0D218C5
:10818000907831003A0000F0AEF800289DD13B888D
:10819000042B03D001213000FFF724FF012C04D170
:1081A000A868002801D003F0F3FC280003F030FC9D
:1081B0008020039B0002434018000DB0F0BD012851
:1081C00000D182E701213000FFF70CFFEDE7C04648
:1081D000F864FF1FE864FF1F010017000B780370AD
:1081E0004B784370CB788A781B02134343807047E7
:1081F0000A88030002700A88120A42700A88012A5B
:1082000006D14A8882704A88120AC27004207047D8
:1082100002208242FBD14A8804309A704A88120AAE
:10822000DA708A881A718A88120A5A71EFE710B5D3
:108230000400012082420CD94B780A781B021343B8
:108240002380834206D1CB788A781B021343638054
:10825000002010BD022BFBD1CB788A781B02134380
:1082600063804B790A791B021343A380F0E70B88E4
:1082700003700B881B0A43704B8883704B881B0A62
:10828000C3708B8803718B881B0A4371CB88837101
:10829000CB881B0AC3710820704703000120082AFD
:1082A00014D14A780878120202431A80CA78887872
:1082B000120202435A804A790879120202439A80D4
:1082C000CA798879120202430020DA80704710B51B
:1082D00004000120022A05D100204B780A781B02F5
:1082E0001343238010BDF8B5060010200F001500C1
:1082F00003F03EFB04000120002C0ED0A0230C2232
:10830000290023806780201D002D07D003F0C8FBC3
:108310002100300003F0ECF90020F8BD03F078FAFA
:10832000F6E7F7B51E00009008AB142017001D7883
:10833000019103F01DFB041E12D0A2230370019BC8
:1083400047704380099B057146710C220830002B51
:1083500007D0190003F0A4FB2100009803F0C8F92E
:10836000F7BD099903F054FAF6E737B5041E0FD0AC
:108370004388002B0CD00025C1881323007A1722D4
:1083800001950095FFF7CDFFFF236580637225708F
:1083900037BD000010B50C4904004A88002A09D0F6
:1083A0008B89002B05D00020CB8A0222834201D08A
:1083B00010BD012213000A20434300204032C8545C
:1083C000C81842800472F3E7CA64FF1F0023438089
:1083D00003707047094B00211A0010B55C88002C0F
:1083E00006D01C79844203D10A234B43D01810BD18
:1083F00001310A330329F1D10020F8E7CA64FF1FD5
:1084000010B50400407A03F0EBF9FF23637210BD4E
:108410007047043010B580B203F0DAFA002803D0B8
:108420000421494203F05CF910BD000070B500253D
:10843000104CA0682580A581A580A84202D003F039
:10844000A7FBA56000250C4C0C4B606D1D80230024
:1084500058331D70A84202D003F09AFB65650025D1
:108460006068002801D003F093FB013508340A2D21
:10847000F6D170BD9065FF1F3465FF1F8465FF1F37
:1084800070B5041E09D1054D2880A881A880A86870
:10849000002802D003F07CFBAC6070BD9065FF1F2C
:1084A000F0B54B8885B00193002343600A7905003D
:1084B0000F00022A00D07BE0CA88032A17D98B68F4
:1084C0005E7819783602DC78D8790E4399781B7A71
:1084D00024021B020C43034353495BBA0B80331D38
:1084E00093421ED1042C04D0631F022B0ED901200D
:1084F00015E0019A4D4B1201D35A002B06D001987A
:10850000FFF7BEFF4A4A1369013313610421B868BB
:108510002E812C80494203F0E3F86860002005B00A
:10852000F0BD434D042C06D0631F022B0FD9EB681E
:108530000133EB60DBE7019A3C4B1201D35A002B6D
:1085400005D00198FFF79CFF2B6901332B61374B56
:1085500030000293019B029A1B01019300230199B1
:108560008C468B52130063449C8003939E81FFF7DB
:1085700050FF039B041E986016D00421B86849423E
:1085800003F0AEF8FA880100043A200003F088FAFC
:108590000199029AFB888A5A043B9B18029A8B52D3
:1085A0002B6801332B60A2E7AB690133AB619EE717
:1085B0001E4B0293019B1E01029BF35A002B2DD0F0
:1085C00002998C19A068002828D0012A26D1FA889F
:1085D0009B189BB27352A189994217D39B1AC0185A
:1085E000B96803F05DFA029BA289F35A934200D066
:1085F0007DE700222B81A3882B80A3686B60029B00
:10860000F2520B4A53680133536070E7084A93688B
:10861000013393600198FFF733FF68E7044A536919
:1086200001335361F6E7C046FA64FF1F9065FF1FF0
:108630000065FF1F70B5051E15D10B4C0B4B188044
:10864000230058331870606D002802D003F0A0FAA0
:108650006565250050356068002801D003F098FA60
:108660000834AC42F7D170BD3465FF1F8465FF1F2D
:10867000F0B51700A12285B0920001934243394B17
:1086800006001B680C009B18D933FF331D78FDF7DB
:1086900041FF0430854204DD3000FDF73BFF04302C
:1086A000C5B2BD4207D33A0000213000019B03F060
:1086B000DFF905B0F0BD2900380003F021FA2300EE
:1086C000C6B250331E700393019B290063653800C6
:1086D00002F0E6FFCBB20293002B02D0039B0136DF
:1086E0001E7000262300503303931B78B34204D836
:1086F000606D002831D10020DBE7029A2800002AB3
:1087000004D0013B1000B34200D02800F700E71965
:10871000387003F095FA786000280ED03A78019905
:1087200003F0BEF9019A3B780136D3180E4A019343
:10873000D369F6B20133D361D4E7039B1870606547
:10874000A74205D1084A1320D36A0133D362B0E7A8
:10875000606803F01DFA0834F2E703F019FA002309
:108760006365C8E73409FF1F0065FF1FF7B50D00FB
:1087700007000421686802F0B3FF2B89040003702E
:108780002B891B0A43702B8883702B881B0AC370AC
:108790002E8902250436F6B2F42E15D81B4B9F42C3
:1087A00014D10C2003F0E4F81135011E0CD09023F5
:1087B00003708E3B0371043B4380154B8460C6807D
:1087C000187802F095FF00252800FEBD5C237B434E
:1087D000104AD3180093583301931B78002B0FD104
:1087E0000300320038000099FFF742FF019B0500AB
:1087F0001B78002BE8D13800009903F069F9E3E712
:10880000054A0725536A01335362DDE7FEFF000086
:10881000F864FF1F3465FF1F0065FF1FF0B587B0C8
:10882000009017200F0016000193FFF7F2FD1325AB
:10883000041E19D00C98031E02D00199201D9847E0
:10884000030AE370052302AAA07004309081277008
:108850000098667003A993800494FFF787FF051EB4
:1088600002D0200003F094F9280007B0F0BD00000A
:10887000F0B587B01F000CAB1B7803910593012165
:108880000DAB06001C78049200F0D6F814250028E1
:1088900021D02000FFF77EFD0135041E1BD01149B9
:1088A000059B0A7803700132D2B2131EC68001D133
:1088B00001231A000B7022713000049B039900976A
:1088C000FFF7ACFF051E09D1230021000648074A27
:1088D000093302F0E5FF280007B0F0BD00236380F4
:1088E0002370F8E7FC64FF1F6B83001130750000F4
:1088F000F8B505000E00064C064F2368002B02D089
:108900003100280098470434BC42F6D1F8BDC04677
:10891000A065FF1FB465FF1F0123064A5B42538019
:10892000002313715362044A136053609360D36051
:1089300013617047B465FF1FA065FF1F020000238D
:1089400010B506499C000859002801D1625010BD9D
:108950000133052BF6D11320F9E7C046A065FF1FB0
:10896000034A5388181A4342584140421040704706
:10897000B465FF1FF0B585B002930AAB1F780CAB4E
:108980001B88009008000E0001920393FFF7E8FF98
:1089900005001120002D1BD10E48FFF7E1FF040058
:1089A0001520002C14D006220B99A771E01D03F0AE
:1089B00077F8019B30002371029B29006371009BB3
:1089C00066802370039B6562E381FFF791FF2800B7
:1089D00005B0F0BDFFFF000010B5FFF7C1FF0400B8
:1089E0000220002C12D060880121FFF781FF606A0D
:1089F000002801D002F08CFE28220021200002F085
:108A000007FF012300205B426380207110BD00003E
:108A100030B5074A074C5588010013780020A5425D
:108A200004D05B1A59424B415842104030BDC046F9
:108A3000B465FF1FFFFF0000084A10B501230C00BA
:108A4000904208D0FFF78CFF031E04D00379234027
:108A50005A1E9341DBB2180010BDC046FEFF000055
:108A6000024B1879431E9841C0B27047B465FF1F8E
:108A700070B504000D001600FFF772FF002804D146
:108A80000D4B9C4200D0143070BD416A0379052023
:108A9000002907D012221A40102A02D10520002EE8
:108AA000F2D10F20DB06EFD5897E0C20A942894147
:108AB000494249420840E7E7FEFF0000030010B5C5
:108AC000002800D110BD0348034A41889142F9D0E3
:108AD0009847F7E7B465FF1FFFFF0000002330B59C
:108AE000C45CCD5C6C40D4540133102BF8D130BD44
:108AF0000F23002210B5C45C64002243CA54C25C38
:108B0000D209013BF7D210BD0200010010B520329E
:108B1000103102F045FF10BDF0B58BB0039010206E
:108B200005931700049102F01BFF0090102002F043
:108B300017FF009B13240190002B05D000280CD1B7
:108B40001324009802F0E4FD019B002B02D01800D2
:108B500002F0DEFD20000BB0F0BD102002F000FF9F
:108B60000600102002F0FCFE13240500002E00D1A8
:108B7000AEE0002819D01022002102F049FE320098
:108B80002900039802F00CFF041E0ED133787F2BCE
:108B900051D830000099FFF7ABFF009B1B787F2B6B
:108BA00053D801990098FFF7A3FF300002F0B0FD01
:108BB000002D02D0280002F0ABFD002CC1D1102006
:108BC00002F0CEFE0600102002F0CAFE0290002E37
:108BD0007CD0002878D03A000F32230001251211F2
:108BE00005D00F333B4015B25A4253411BB26A1EA7
:108BF0001201002B33D0049BD2B298180099029A2C
:108C0000FFF76CFF013D10220021300002F000FE52
:108C1000ADB2049F2D017D19AF4242D0002C33D05C
:108C2000300002F075FD029B002B00D189E718008F
:108C300002F06EFD85E729003000FFF759FF28009C
:108C40002549009AFFF74AFFA7E729000098FFF798
:108C50004FFF28002049019AFFF740FFA5E70F21A9
:108C60000F4004998A18D9B28F4208D9D15C06A85E
:108C700019540133102BF6D1029A0199C0E7791AE1
:108C800048424141C901F2E73900300006AAFFF726
:108C900025FF3200039806A902F082FE1037040077
:108CA000BAE7002CBCD13000029906AAFFF716FFE4
:108CB000320006A9039802F073FE08220400310076
:108CC000059802F0EDFEABE71324A9E71324AAE709
:108CD000002800D06EE733E790BE0011F0B58BB0EE
:108CE0000F0016000225009000283FD0002A3DD03A
:108CF0000B1DDBB21800029302F032FE1135041E88
:108D000034D0FDF747FD05003A000099201D02F020
:108D100097FCEBB20393E3702B0CDBB22F0A0093AA
:108D20006370FFB22B0E2370A7700193FDF72CFD2B
:108D30001022010006A802F083FC2100029A04AB75
:108D400006A8FFF7E9FE051E0DD1039B082233702C
:108D5000009B04A9B370019B7770F370301D02F083
:108D60006FFCFDF71DFD200002F0D2FC28000BB0C7
:108D7000F0BDF0B58FB00D00149E039004920593E2
:108D8000002A03D1022420000FB0F0BD002EF9D03C
:108D90000398FFF7E5FD1424071EF4D072783378AA
:108DA00012021A43B3781B041343F27812061A43D3
:108DB000036A0192934201D30133E3D1002D03D022
:108DC0003B7901249B07DED50822002106A802F08A
:108DD0001FFD059B13240433DBB21800029302F03D
:108DE000BFFD051ECFD0059A0499043002F028FC7F
:108DF00004223100280002F023FC39001022103137
:108E00000AA802F01DFC2900029A06AB0AA8FFF787
:108E100083FE041E0FD1082206A908A802F010FC48
:108E20000822311D08A802F0ABFE012807D10199E4
:108E30000398FDF7C9FC280002F06AFCA3E70124AF
:108E4000F9E7000070B51C4C05002368181E10D00F
:108E5000002D14D11A78002A0CD1981C083202F087
:108E60001FFE02F035FD0135002808D123681D7072
:108E7000012070BD0A331800082202F011FE236899
:108E8000002BF5D0122002F073FD061E0DD0C12379
:108E900021680370457002311022023002F000FE9A
:108EA00023683100587802F023FC206802F030FC7F
:108EB00000232360DCE7C046DC65FF1FF8B5040033
:108EC0002020FDF755FB0D4EA700BB590500002BD8
:108ED0000DD000280BD0D878FF2809D108492A00E6
:108EE0000C55F35907480333611802F0D9FCF8BD5B
:108EF000290002F07DFB0028F0D1F8E7F865FF1F9C
:108F0000E065FF1F15A1001170B5064D840063597F
:108F1000002B05D0D87802F063FCFF226359DA7089
:108F200070BDC046F865FF1F70B506008CB00C0020
:108F3000150000213022684602F06AFC3100102240
:108F4000684602F07DFB1D2021000322684402F0E8
:108F500077FB6846FFF7D8FD2D2104000322280087
:108F6000694402F06DFB20000CB070BDF0B5070045
:108F7000160097B001931CAB1D7830221EAB0091F8
:108F80000AA800211C7802F043FC102239000AA82C
:108F900002F056FB1022002102A802F039FC072241
:108FA000310002A802F04CFB072202AB9818631EA6
:108FB0009C41019902F044FB02AB9C732B005A1EAA
:108FC000934102AAD3730021102206A802F020FCCC
:108FD00006221D9907A802F033FB1A2002ABC01825
:108FE00006221F9902F02CFB102200990EA802F015
:108FF00027FB102202AB0EA908781C78013A6040CA
:10900000D2B2087001330131002AF5D10AA8FFF766
:109010007BFD102212A904000EA802F041FD1022CF
:1090200006AB0EA908781D78013A6840D2B20870E4
:1090300001330131002AF5D10AA8FFF765FD044389
:1090400010222098E4B212A902F0FAFA200017B018
:10905000F0BD70B50E0014008CB0010010226846FF
:109060001D0002F0EDFA3100082204A802F0E8FA2F
:109070002100082206A802F0E3FA6846FFF744FD43
:1090800004001022280008A902F0DAFA20000CB02F
:1090900070BDF8B506000D0000243719AC4200D3AE
:1090A000F8BD02F06DFC030A3B70631CDBB20137B4
:1090B0009D4203D90234F054E4B2EEE71C00EDE720
:1090C00073B506000C000225002819D0002917D01E
:1090D000032101A8FFF7DDFF6B469A793F231A4071
:1090E000013313436A463000937101A92200FFF750
:1090F0001BFF051E04D10322E01C01A902F0D0FCD5
:10910000280076BD03785807DA08C00FD200800027
:109110009B0710439B0F1843C0B2704707230B40B7
:10912000C908C9000B4303707047000070B5040004
:10913000FFF7EAFE134DA4006359002B21D0186AF3
:10914000002801D002F0E4FA2B59986E002801D0D3
:1091500002F0DEFA2B59D86E002801D002F0D8FABE
:109160002B59186F002801D002F0D2FA2B59586FF2
:10917000002801D002F0CCFA285902F0C9FA0023E5
:109180002B5170BDF865FF1F0E4B8000C35870B5A2
:109190000C00002B0FD09D68002D0CD02B78201DCB
:1091A0000B706B784B70A97CFFF7B8FF2B7E237296
:1091B0006B69E36070BD10220021200002F028FBE3
:1091C000F8E7C046F865FF1F014B18607047C046BE
:1091D000F465FF1F074A03008000825810B5002A7B
:1091E00006D0D088984203D1012901D1FFF79EFF14
:1091F00010BDC046F865FF1FF0B5264E95B087003C
:109200000B93BB590500099112200A92002B31D013
:10921000D888FFF7A5FB04001420002C2AD02800D2
:1092200010A9FFF7B1FFBB591E781D6A002E23D08D
:109230000895FDF7EFFA07000020FDF7F1FA079017
:10924000A379E61D069310AD0CA9089800F0E2FA88
:109250000EA9280000F0D7FA0B9B0A990493069BED
:1092600009980293079B0396019300970EAB0CAAF3
:10927000FFF77CFE15B0F0BDFDF7CCFA069030008C
:10928000FDF7CEFAE31DA779079310AB060008930C
:10929000DAE7C046F865FF1F30B50C4C85002A5947
:1092A000030085B00120002A0ED018006946FFF7A0
:1092B0006BFF2B591A78D888054B002A00D1054B33
:1092C0006A46072100F0D9FB05B030BDF865FF1FE5
:1092D000079800111598001130B5094C85002959DF
:1092E00085B010226846253102F0DAFB2A59112197
:1092F000044BD0886A4600F0C0FB05B030BDC046C4
:10930000F865FF1FB198001130B5094C8500295947
:1093100085B010226846353102F0C2FB2A5911216E
:10932000044BD0886A4600F0A8FB05B030BDC046AB
:10933000F865FF1FEF980011F7B54D4F860010201C
:10934000F4590D0002F00CFBF3592062186A132245
:1093500000286CD0033A29009C6802F0A1FBF35965
:109360001A780192002A58D11E6A227D317B9446D8
:1093700051400122019F114201D167461740217DD2
:10938000914339432175377B4F40BC4660460027E7
:10939000800701D44F081740012102208F40227D11
:1093A00082433A432275377B5740BC4660460027CC
:1093B000400701D497080F400420227DBF0082435C
:1093C0003A432275627D002794466046727B424094
:1093D0000A4201D167460F400121627D8A433A4328
:1093E0006275777B5740BC4660460027800701D4F2
:1093F00057080F400220627D7F0082431743677544
:10940000767B00227E40760701D4BA080A40042603
:10941000617D9200B1430A4362756A78002A08D0E0
:109420006278002A05D005220533DA770022100081
:10943000FEBD04222979114205D1A17C114202D13D
:109440000533033AF1E7019A21782C78002A02D1FA
:109450000A002100140018220429E8D8042CE6D8B8
:1094600005206043034A05331218525CDDE7C0460D
:10947000F865FF1FA0BE001110B50A001121024BB4
:1094800000F0FBFA10BDC0464B9900110B0030B53F
:1094900087B001AD2B806B4604001100981D082297
:1094A00002F0FEFA2A000B212000024B00F0E5FA40
:1094B00007B030BD7399001110B50A001121024B9D
:1094C00000F0DBFA10BDC046C799001113B50B00C0
:1094D00011006A4613706B4604000622581C02F005
:1094E000DFFA6A4608212000014B00F0C6FA13BDDE
:1094F000E799001110B50A001121024B00F0BDFAE6
:1095000010BDC046379A00117FB505000B4BAA006D
:10951000D4580800002C0FD0666F237FE288217892
:109520000396266F0296E66E0196A46E0094FDF7F0
:1095300009FC2800FFF7FAFD7FBDC046F865FF1F54
:1095400010B51721FFF7E0FF10BD000070B50A004D
:109550000D00064B0221040000F08FFA0600297866
:109560002000FFF7D1FF300070BDC04617990011F1
:1095700070B586B000236A461370836804001D78B6
:10958000681E0A2859D801A902F04AFA060633379C
:109590003B3F43474B4F5300180000F042F906236E
:1095A00012284BD000281BD16088FFF7D9F9082377
:1095B000002813D04279002A47D1264B1A78072376
:1095C00012070BD5244B1A680723002A06D0166809
:1095D000002E03D0290001AAB04703006A46137089
:1095E0006B461B786088002B2AD1FFF767FC06B01A
:1095F00070BD180000F06CF9D4E7180000F087F98E
:10960000D0E7180000F093F9CCE7180000F0ADF9AE
:10961000C8E7180000F0C3F9C4E7180000F0F6F935
:10962000C0E7180000F0F6F9BCE7180000F013FAE4
:10963000B8E7180000F013FAB4E707236A4613707E
:1096400069466088FFF782FFD1E70523012AC5D16B
:10965000024BB8E78564FF1FF065FF1FF465FF1F2D
:10966000F8B52C4F8600F35904000D00002B40D0B4
:10967000DA8882423DD15A78062A33D11A78002AF4
:109680002ED0012099681A6A097D014206D0157B07
:10969000054203D007225A700120F8BD0220014282
:1096A00004D0157B054201D00922F4E704200142D1
:1096B00004D0127B024201D00B22ECE7164B1B6850
:1096C000002BE9D05B68002BE6D020009847BB59FF
:1096D00000215B78122BDFD12000FFF715FFDBE7BD
:1096E0000E4BECE7112A04D1002900D032252900C5
:1096F000F2E7002D08D12000FFF732F9002803D04F
:10970000102302791343037121002800FDF798FA12
:10971000C2E7C046F865FF1FF065FF1FF465FF1F35
:1097200070B50E4E8500AB590400002B13D01B788A
:10973000002B11D10A4B1B68002B04D05B68002B57
:1097400001D02000984773595B78122B03D1002178
:109750002000FFF7D9FE70BD024BECE7F865FF1F54
:10976000F465FF1FF065FF1F094B8000C3581020F0
:10977000002B0CD01A6A002A09D09B68002B06D057
:10978000127A1B7E101C9A4200D9181CC0B2704776
:10979000F865FF1F70B503000D0014000220002AB9
:1097A00030D000292ED013700B78081D53704B78E1
:1097B0009370FFF7A7FCE070012002212B7A237140
:1097C0006B7B034063716A7B0A401343042263711D
:1097D0006E7B1640334363716E7BF608F6003343AD
:1097E00063712B7B0340A371287B014000200B4356
:1097F000A371297B0A401343A3712A7BD208D200AC
:109800001343A37170BD10B50A0001000120FFF7DA
:10981000C1FF10BD10B50A0001000220FFF7BAFF1A
:1098200010BD70B506000C000220002E30D00029BB
:109830002ED07378201D0B70B3784B70F178FFF742
:109840006DFC01223579257271794B1008001340A7
:10985000934010400343881010408000C908034320
:10986000C9000B436373B1794B1008001340934058
:1098700010400343881002409200C9081343C900F6
:109880000B4321202373FCF773FE854201D2122083
:1098900070BD2220257AFCF76BFE8542F7D823782D
:1098A0001820042BF4D86378012BF1D80020EFE7BF
:1098B000030010B50220002909D0002B07D0032295
:1098C000481C0A7019000D3202F0EAF8002010BDA1
:1098D00003000222080010B5002B06D0002904D096
:1098E0000E32591C02F0DCF80022100010BD0300FB
:1098F00010B50220002909D0002B07D00422481CF3
:109900000A7019000C3202F0CBF8002010BD10B51F
:10991000FFF7DEFF10BD03000220002906D0002B58
:1099200004D0052200200A701B784B70704703009A
:109930000220002B08D0002906D05B7800200B7095
:10994000013B082B00D918307047030010B50220E6
:10995000002909D0002B07D00622481C0A701900E4
:109960000A3202F09DF8002010BD10B5FFF7B0FFDD
:1099700010BD02000B00022010B500290ED0002AF5
:109980000CD007211970118859701188090A997033
:1099900011180822D81C02F083F8002010BD030023
:1099A0000A00022010B5002B0CD000290AD09978AB
:1099B0005878090201431180901CD91C082202F03A
:1099C0006FF8002010BD030010B50220002909D057
:1099D000002B07D00822481C0A701900921802F0C8
:1099E0005FF8002010BD02000B00022010B5002916
:1099F0000BD0002A09D00921197011781818597054
:109A0000511C062202F04CF8002010BD10B5FFF7E3
:109A10005FFF10BD02000B00022010B5002A09D024
:109A2000002907D05178197011180622581C02F02D
:109A300037F8002010BD030010B50220002909D01E
:109A4000002B07D00A22481C0A701900063202F0C7
:109A500027F8002010BD10B5FFF73AFF10BD020037
:109A60000B00022010B5002A06D0002904D01800EF
:109A70005178FFF753FB002010BDF0B585B01700FB
:109A80001E006A4606230500080091819380FEF7B8
:109A9000C0FC1324011E02900CD03800B047041EF5
:109AA00005D1280001A9FEF76FFA041E02D0029822
:109AB00002F06EF82800FFF701FA200005B0F0BDB3
:109AC000F0B504008BB0019115000021102202A80E
:109AD00001F09EFE334EA700B85900283CD0C38841
:109AE000A34239D10378002B36D14278062A18D107
:109AF00002000100553235310C3006ABFFF7A9FAF0
:109B0000002829D12000FFF72FFE020006A902A895
:109B100001F0C6FF200002A901F072FD01200BB088
:109B2000F0BD816E002917D00B8A112A28D19D42E1
:109B30000ED101981231093A02F022F8012807D11A
:109B4000BB5920009D6EFFF70FFE29000200DEE7E3
:109B500032212000FFF7D8FC2000FEF701FF061E8F
:109B60001BD0416A002918D00B8AAB4215D10822BC
:109B70000198123102F004F801280ED1716A0AE04E
:109B80009D42E9D108220198123101F0F9FF012824
:109B9000E2D1BB59996E8A7EB9E7200001F0F8FD49
:109BA000BCE7C046F865FF1FF0B56B4D87007E59D6
:109BB00085B0337802900393002B00D087E0B36820
:109BC000346A01937078062817D101221B7D134255
:109BD00002D0217B114218D10222134202D0217BF4
:109BE000114251D10422134203D0237B134200D0EF
:109BF0008BE0019B5A7DEB5991E007380428F8D897
:109C000001F00EFF032E42678300B36E002B03D1D9
:109C10001C2001F0A5FEB066EB599C6E002C1CD0F8
:109C200010220021200001F0F3FD0298FFF79CFDB7
:109C300001002000FFF72DFA01F0A2FE2082200093
:109C400008211230FFF725FA0298FFF78DFDA07664
:109C5000EB592100D888FFF70FFC0822EB591CE0D4
:109C6000B36E002B05D01A00198AF0881232FFF764
:109C70000DFC0222019B197DEB5911423DD0207B46
:109C800010423AD0073208E0F488FCF7DBFD01000F
:109C90002000FFF711FC0A22EB595A70029B9C002E
:109CA0002A595378073B042B11D8D088FEF758FE69
:109CB00000284ED0C3895A08D2182849029B02981E
:109CC000CB542B5941180433254801F0E9FD05B068
:109CD000F0BDFCF79FFD03000120834201D100206D
:109CE0000393EB59DE88FCF79BFD039902003000DB
:109CF000FFF7ECFB019AEB59117D042211420CD0C5
:109D0000217B114209D00B22C7E7F688FCF73CFD06
:109D100001003000FFF7EEFB6BE7019A527D012155
:109D20000A4204D0607B084201D00C22B5E7022130
:109D30000A4204D0607B084201D00E22ADE7042124
:109D40000A4204D0627B0A4201D01022A5E7122207
:109D5000A3E7FA225200B0E7F865FF1FFC65FF1F7A
:109D60001FA1001110B5064B1A78042310001840EB
:109D70001A4200D00348FFF727FA002010BDC04662
:109D80008564FF1F4843FF1F70B50400FFF7D4FA36
:109D9000051E43D12000FFF77FFA234EA400A059EF
:109DA0008268937CDB0708D50321036A1B790B408B
:109DB000012B02D1017F0B430377431DD97F8B1EFB
:109DC000022B0DD8022900D00121C088FCF790FF9A
:109DD000042133591A7F59700A431A77280070BD3D
:109DE00001290CD102231022437000210C3001F014
:109DF0000FFD305910213530FFF74BF9EEE70529FB
:109E0000ECD10223D118437010220C3001F048FE2F
:109E100004233259117F0B431377EAE708251828EA
:109E2000DCD1053DDAE7C046F865FF1FF0B58BB021
:109E3000059143887E4F9E00F45915000493002C31
:109E400015D1012902D000200BB0F0BD101D5778AC
:109E50001678FFF757F9EB68320002932B7A0499D2
:109E6000019300903B002000FCF70CFFEBE7E38838
:109E7000049A934201D00820E6E72378012B00D111
:109E8000D4E0059B581E092800D9CFE001F0C8FD99
:109E900005CE0A29CC506C859AB229000498FFF7A8
:109EA00073FFD1E7200029001022453001F0F8FDB2
:109EB000B9594B78042B02D1013B4B70C3E70B001F
:109EC0000A00253335320C310498FFF795F90498D0
:109ED000FFF702FA0522431E9841BB59C0005A7091
:109EE000B2E7200029001022553001F0D9FD049B73
:109EF0004F4C9D00295904980A0006AB55320C318D
:109F0000FFF77AF929591022453106A801F038FEE9
:109F1000012808D10498FFF7F7F90590002804D12B
:109F200006222B595A7005988EE708230593FAE705
:109F300063780C2B7AD1E36E002B03D11C2001F047
:109F40000FFDE066BB59D86E00286FD010222900A3
:109F500001F0A6FDBB590498DC6EFFF705FC0D224D
:109F6000A076BB595A706EE7E06E00285ED0637829
:109F70000D2B5BD12B8808220382A91C123001F023
:109F80008FFDBB599A68517D0222114226D0186A72
:109F9000407B104222D00C32E4E763780E2B45D18F
:109FA000236F002B03D1162001F0DAFC2067BB5988
:109FB000186F002803D01022290001F071FD0F2234
:109FC000BB59CFE763780F2B30D1206F0622691C75
:109FD000103001F065FDBB599A68517D0422114291
:109FE00003D0196A497B1142D5D100210498FFF7AB
:109FF0008BFA28E7636F002B0DD0BB59586F0028F0
:10A00000F3D01022290001F04BFD0122BB5952422E
:10A010005B6F1A61E9E7142001F0A2FCBB5960678D
:10A020005B6F002BE9D126E72978DFE707200BE7F4
:10A03000F865FF1F10B5064C207001F009FC0621E1
:10A040002078FDF791FF0348FEF778FC10BDC0466D
:10A050000B66FF1FD591001100200BB270B50D00EB
:10A06000834216DA264B187801F07AFB041E0DD0D5
:10A070000378922B0ED0A02B37D0224B1878FF28D4
:10A080003AD0210001F034FB002835D180200002B5
:10A09000684070BD43780E2B0BD03E2BEDD18378FA
:10A0A000052B12D0082BE8D181798088FFF7D8FAE8
:10A0B00008E0154B82889A42DFD183681878591CD2
:10A0C000FEF7C0FE002817D1D7E7104B1B785B07BF
:10A0D00012D50F4B1B68002B0ED09B68002B0BD0AA
:10A0E000C289811D80889847ECE7FFF741FAA06894
:10A0F000002801D001F04CFD200001F089FCC5E7EB
:10A100000B66FF1F4143FF1F182000008564FF1FDF
:10A11000F465FF1F10B50078FFF712FA10BD10B5F7
:10A120000078FFF7FDFA10BD0C234343084A10B531
:10A130009B185A68002A03D0012901D1904710BD0D
:10A140009B68002BFBD00029F9D19847F7E7C04660
:10A150002866FF1F01238340094A10B5946B1C43F6
:10A160009463506B98435063D46B2000984301294B
:10A1700001D120001843D063116B0B43136310BD52
:10A1800000800040F0B500240127154B85B0DA6B44
:10A19000144E03921A6C0192DA64019BE3403B4235
:10A1A00017D0039DE5403D400295E5B20299280095
:10A1B000FFF7BAFF316A736A002908D03900002B13
:10A1C00001D0029979402800FFF7C4FF01E0002B7D
:10A1D000F9D101340C36172CDFD105B0F0BDC046E3
:10A1E000008000400C66FF1F064B01215A68C240E8
:10A1F0000A4204D01B68C3401800084070471B6D1A
:10A20000F9E7C046008000400122064B8240002949
:10A2100003D0D9680A43DA607047D9689143D9609E
:10A22000FAE7C0460038004030B5032444430F4BE2
:10A23000E25C1B199C785D7801232D1B0135AB4036
:10A24000013BA340A140DB430C00122807D808497A
:10A2500092005218116819402143116030BD054A1F
:10A2600011680B4023431360F8E7C046E7BE0011B6
:10A2700008F0004014F00040C21F70B5D4B20623AD
:10A28000092C0BD80125084C9540002908D0002145
:10A29000FFF7CAFF23682B4323600023180070BD1B
:10A2A0002368AB43F8E7C04600380040214BF0B5C7
:10A2B0001B185B78022B21D1032444431E4A1F4EF6
:10A2C000A35C12199478012215008540B76B013CFC
:10A2D000E4B23D43A240B563194C122815D89B0047
:10A2E00000290CD117495B1899680A439A60012329
:10A2F000205C154A834011680B431360F0BD11497F
:10A300005B18996891439960F1E70E4B00290DD1D4
:10A3100059690A435A61225C1328E8D00123203A84
:10A3200093400A49086803430B60E7E75969914382
:10A330005961F0E70C66FF1FE7BE00110080004086
:10A340002CBF001100F00040A0F00040A4F000403D
:10A35000F8B500241B4E1C4D1C4B1B5D012B1FD15F
:10A36000194A9269E2401A420BD00122B256934038
:10A370002200143AD2B2022A09D815494A69134375
:10A380004B61013402360C35172CE5D1F8BD0022A3
:10A39000B2560F499200521891680B439360F0E750
:10A3A000022BEED1E7B23800FFF71EFF0123584021
:10A3B000C1B23800FFF77AFF3800FFF715FF687762
:10A3C000DFE7C046B9BE00110C66FF1F0D66FF1F18
:10A3D00000F00040012202388240054B002903D0E2
:10A3E00059690A435A617047596991435961FAE7BB
:10A3F00000380040F8B50E0001210F008740114AD7
:10A400000400D368FD43BB43D360831E8B4201D855
:10A41000FFF7E0FF00212000FFF72EFF0A4A0B4B59
:10A420005168012E05D139431B1951605E7000201F
:10A43000F8BD2940516002221C1962709A691540CA
:10A440009D61F4E700380040008000400C66FF1F6B
:10A45000012210B58240074B002906D019680A4333
:10A460001A600121FFF7C6FF10BD196891431960FA
:10A47000F7E7C046008000400C2370B50025434339
:10A480000A4A29009B181D70094B04001B185D70B7
:10A49000FFF7B0FF0123A340064928000A681A43CA
:10A4A0000A6005490A689A430A6070BD2866FF1F62
:10A4B0000C66FF1F348000403080004070B50400FF
:10A4C0000E00FF2813D003250540FFF7D5FF084AEB
:10A4D000A3089B009B183F22ED00AA40AE401968DC
:10A4E00020009143314319600121FFF78DFE70BDBB
:10A4F00018380040F8B50C244443134B0500E41809
:10A500006368002B03D1A3681220002B1AD002220B
:10A5100001270E4B00215B195A7028002770FFF7A6
:10A5200069FF63681E1E08D0A3683E00002B04D09C
:10A530002800FFF759FE4640F6B228003100FFF729
:10A5400009FE0020F8BDC0462866FF1F0C66FF1FED
:10A55000F7B5C420FF222B4B8000195800249143EB
:10A560003F3A0A431A508022274F5202274E1A6060
:10A57000274B1D5D002D21D0A31E012B03D80121E7
:10A58000E0B2FFF727FF012D18D11F4B9B69E34075
:10A590002B4213D0E3B218000193FFF725FE010010
:10A5A0000198FFF755FFE3B2143B022B1DD80121A0
:10A5B0007156184A8D405369AB4353613B7F002B62
:10A5C0000DD0E5B22800FFF795FF2800FFF70CFE3D
:10A5D0007B7F0100834202D02800FFF7A5FD0134F4
:10A5E0000C370236172CC3D1F7BD01210023715659
:10A5F000F3568D40074A9B009B189A68AA439A60BD
:10A60000DCE7C04600E100E00C66FF1FB9BE0011A8
:10A610000D66FF1F00F0004010B501210400FFF798
:10A62000E9FE0123044A002011194B70A3409169EF
:10A630000B43936110BDC0460C66FF1F70B50E0042
:10A6400015000400FFF718FF0C236343094A20009C
:10A650009B189D605E60FFF74DFFF021064B074A97
:10A660008900051E5A5002D02000FFF705FF280080
:10A6700070BDC0462866FF1F0000FF1F85A10011A6
:10A6800070B5134D07202C78002C1FD19822210083
:10A690005200280001F0ECF80123C420FF222B70A7
:10A6A0000C4B80001C635C630B4B1C605C600B4BB1
:10A6B000195891433F3A0A431A50802252021A60B5
:10A6C0000D20074A074901F09BF8200070BDC046E5
:10A6D0000C66FF1F00800040A0F0004000E100E099
:10A6E00051A5001151A30011030010B50620072B3E
:10A6F00009D8054A137001F09BF8D7210020034BBD
:10A70000034A89005A5010BD7043FF1F0000FF1F0D
:10A71000D91AFF1F70B51D0002240C2910D8094A50
:10A72000CA40D2070CD5FBF72FFF041E08D1059AAB
:10A7300004992800FBF744FFFCF7B2FDFFF712FB7A
:10A74000200070BD1210000030B50D7802232C00DF
:10A750009C43184201D02B431C0008252300AB4327
:10A76000284201D02B00234320241D00A543204272
:10A7700001D01C4325002A230D70184204D0117803
:10A780001E3B0B43137030BD0028FCD10C21137805
:10A790008B43F7E7F8B51D0006AB1B88140007AA2A
:10A7A0000E000B201778002B27D10A78022A49D1F6
:10A7B0004A68507811780002244A08438018042817
:10A7C00040D801F02DF903121D1B2300F06801F0A1
:10A7D00047F9021CC0B2B84200D93A1CD2B22000DC
:10A7E000F1682A8001F05CF906E00222F3681B8818
:10A7F0002A8023701B0A63700020F8BD0622EEE752
:10A8000001232B80F3681B782370F5E7F368002B96
:10A8100016D008222A801A8822701A88120A6270BA
:10A820005A88A2705A88120AE2709A8822719A880D
:10A83000120A6271DA88A271DB881B0AE371DBE716
:10A840002B80D9E701202B80D7E7C04600D6FFFF39
:10A85000F7B516000A781D0008AB1F880C0001230D
:10A86000022A18D14A685078117800022B4A08430E
:10A87000801803280FD801F0D3F802254439E06886
:10A8800001F0EEF8C0B20723B84204D37B1901935C
:10A89000152B02DD0D231800FEBDE0682A003100F3
:10A8A000C01901F0FDF86B4600209B88E268D05487
:10A8B0001B4B1B68834203D01B68834200D0984720
:10A8C0000023E8E70B23002FE5D1022DE2D17378B6
:10A8D00032781B021343E2681380114B1B68002B74
:10A8E000EED01B68002BEBD00120E8E70B23002FF4
:10A8F000D1D1062DCED12A003100E06801F0D0F888
:10A90000DEE70B23002FC6D1012DC3D1327875337A
:10A91000012AC0D8E3681A70D2E7C04600D6FFFF0C
:10A920001868FF1F70B50C001500072837D801F014
:10A9300077F8041436361B36242E182015290BD828
:10A94000184E16220021300000F062FF220029007C
:10A95000300001F0A5F8002070BD18200229FBD1BD
:10A960001288114B1A80F6E718200829F4D10A0042
:10A970000E48290001F0BCF8EDE718200129EBD1C1
:10A980000B4B10780B49DA69FFF7DEFEE3E718207E
:10A990000129E1D1064B10780749DA6BF4E7022070
:10A9A000DAE7C0460068FF1FEE43FF1FE443FF1FC6
:10A9B0007443FF1F9C43FF1FBC43FF1F030010B5E0
:10A9C0000020DB0704D50721024A034800F08CF879
:10A9D00010BDC04644BF00117443FF1F054A030069
:10A9E0001068002803D082889A4201D1806870479D
:10A9F0000068F6E7106AFF1F0A88030008009A4201
:10AA000004D08A8804309A4200D0002070470000A9
:10AA1000F8B5F22200230D4F0D4E79680500424330
:10AA20003370994200D07B600A4C0021200000F076
:10AA3000EFFE00231A007C60AB4202D1002033708D
:10AA4000F8BD01332280DBB2F234F5E7086BFF1F5B
:10AA5000066BFF1F146AFF1F73B56B46019006005B
:10AA6000684615001980FCF74DFF041E11D1002D1A
:10AA70000FD07689002E11D00C2000F071FF002835
:10AA80000ED0084A0460136886808560002B02D1CE
:10AA90001060200076BD1A001B68F7E70224F8E773
:10AAA0001324F6E7106AFF1F012100220A4B10B59C
:10AAB00049420A4C198099809A719A70084B20700B
:10AAC000012019805A60FFF7A3FF2078FCF778FF78
:10AAD0000448FDF733FF10BD2068FF1F106BFF1FF8
:10AAE000086BFF1F95AB0011022310B5002802D0A0
:10AAF000FFF7B2FF0300180010BD0000030010B5FF
:10AB00000020DB0704D50421024A0348FFF7A4FF15
:10AB100010BDC04658BF0011F443FF1FF0B50E260C
:10AB200087B003930CAB1F8802ABF6180500080032
:10AB300031000292FDF768F804000120002C0FD0CC
:10AB40003088FFF74BFF03000E20002B08D05E6813
:10AB5000002E05D021002800039B029A0097B047E1
:10AB600007B0F0BD0A4B10B5984207D1012200236F
:10AB700052420A808B708A808B7110BDFFF73CFFB8
:10AB80000028FAD001235B42038000238370F4E79E
:10AB9000FFFF0000F8B5050001290AD1134E00247B
:10ABA0003388F227AB4219D028001149FFF7DAFFAA
:10ABB00006E0022904D10139FDF73EFF0028EDD05F
:10ABC000F8BD3B0063437268D018D35A002B09D0FC
:10ABD0003A00002100F01CFE0134E4B2054B1B7862
:10ABE000A342EED801235B423380DDE7086BFF1FF1
:10ABF0002068FF1F066BFF1F10B5FFF7FDFE030067
:10AC00000020834200D0987810BD0000F0B589B0D4
:10AC10001C000EAB80CB03901E8810AB1B780492F7
:10AC200002930B7A0D00DB0616D42B780593022BCA
:10AC300024D00498FFF7D2FE002812D003689C4667
:10AC4000002B0ED0029B2200019329003B0064469A
:10AC500003980096A04705E00498FFF7BFFE002880
:10AC600002D10E2009B0F0BD8368002BF9D00A2272
:10AC70002900039898470028D7D0F3E76B685878E5
:10AC80001A786B4B000210439842D2D8043B98428A
:10AC900010D2684B984242D015D8674BC018012893
:10ACA000C7D80B20002EDDD1EB681A7859683A809E
:10ACB000200028E0614BC018032800D979E000F09B
:10ACC000AFFE846A789E5E4B9842B2D10B20002E74
:10ACD000C8D101233B80EB6831001B782370688961
:10ACE000013080B2FCF790FF3A88031E0ED0017845
:10ACF00002328A183A80428962704289120AA2702E
:10AD000059680278E01C00F0CBFE06E004323A807D
:10AD100031000422601C00F07BFD0020A2E70B2024
:10AD2000002E9FD1EB6807A91E8804233B80330ABD
:10AD3000300026706370FCF767FF051E28D004AB57
:10AD40009A890E2304A95B183E49C668FCF7D0FF18
:10AD500000280BD12B783C486A680599FBF786FBE5
:10AD6000002803D1012304AA5B42D3813278022A4E
:10AD700006D17168201D00F093FE3B8802333B80B2
:10AD80000E2304AA9B181B88A3701B0AE370C4E758
:10AD900004ABDE81F4E70B20002E00D062E7E96807
:10ADA0000398FFF729FF02233B802070000A6070A0
:10ADB000B3E70B20002E00D054E70222EB681B887B
:10ADC0003A8023701B0A6370A7E7E86800F048FE2A
:10ADD000C2B203000720B24200D243E70DD002996D
:10ADE000DBB27118994202DB921BD3B20293029B31
:10ADF000E9681A003B8089195AE70023F6E70B201F
:10AE0000002E00D02EE70722EB683A801A782270D5
:10AE10005A7862705A88A2705A88120AE2701A79B7
:10AE20002271DA886271DB881B0AA37175E7C0465C
:10AE3000042900000228000000D8FFFFFFD6FFFF12
:10AE400003280000FFFF000088BE0011F0B58DB0A0
:10AE50006B460020089120229B5E83423DDAA64B80
:10AE6000187800F07DFC071E32D00378B02B2CD16F
:10AE70000079023816281FD800F05AFE17001E006D
:10AE80001E001E0031001E0096001E001D011E0047
:10AE900052011E0073011E00CD011E0050021E0053
:10AEA0001E001E008E021E00E302944B94491B8874
:10AEB00078880B80FBF71AF83800FCF79BFF914B62
:10AEC0001B68002B01D038009847380000F0A0FD27
:10AED0008020089B0002434018000DB0F0BDEE2218
:10AEE0000021874800F094FC0BAA3B7B79893889C4
:10AEF00000923A000D32FCF79FFD0400804B1B7856
:10AF0000002C3FD146E0804B788805937F4B410071
:10AF1000CB5A0BAE073BDBB232880293002301937E
:10AF20007B4B210006930093059BFFF76FFE744D4A
:10AF3000002810D1069B3A8A1B889A420BD1380010
:10AF40000599123000F01CFE002804D02B7862898D
:10AF50009B00EB185A80162306A81B183288200085
:10AF60007989FCF7C5FE2B7804009A00AA1851884D
:10AF70000029C3D00133DBB22B70002807D006A90B
:10AF8000C98A9180634A12889A42BCD802E00121A2
:10AF900049429180002B04D059497888FAF7DAFFAA
:10AFA0008AE73E890A2479E000253E89574B0693BB
:10AFB0007B88069A5B009B5A033B9D4202DB002D77
:10AFC000F0D05BE0162206A812183B7B798900922C
:10AFD0003A0030000D32FCF72FFD0590002858D0C4
:10AFE0004689017A7888FCF7F1FC041E44D1464B6F
:10AFF00078880793069B4100C95A454B0439C9B26A
:10B0000006AAD28A06930291019400930599079BA0
:10B01000FFF7FCFD041E2FD1069B39491A88931CAB
:10B02000002D26D14B807988384B4900CB5A5119D5
:10B03000033B8B4220DD059B31485B8941190B7135
:10B04000A91C0135C9B2EDB2059145191B0A2B7136
:10B05000059B2D490433181800F022FD2C4B059A4E
:10B060001B88D318DDB22C4B9E4205D00136B6B2F8
:10B070009CE749889942D6D0002D0CD0204C28005E
:10B08000618800F08DFB207021007888FAF772FF4C
:10B0900012E7059CF0E7002C00D183E77B78142BA6
:10B0A00000D109E716493B794E800B700C71788806
:10B0B000FAF712FF00E7162406ABE41821003889DE
:10B0C000FCF7A2FD011E00D1B7E1788822880F4C61
:10B0D00045002C5B0A4D013CE4B2029400240F4B66
:10B0E00001940095FFF792FD041E00D014E12900A1
:10B0F0007888FAF74FFFDFE6106BFF1FE042FF1F73
:10B100002868FF1F1C68FF1F1C69FF1F5864FF1F72
:10B110000C6AFF1FDE42FF1FFFFF00002A68FF1FAF
:10B12000162406ABE41821003889FCF76DFD011EDA
:10B1300000D182E178882288AE4C45002C5BAE4D70
:10B14000013CE4B202947C89AC4B01940095FFF77A
:10B150005DFD041E00D0DFE029007888FAF724FFA7
:10B16000AAE60025A44B1D803B00F6331B78A24ABB
:10B1700078880792AB4208D99E4B128806930699AD
:10B1800043005B5A013B9A4203DB0799FAF716FF2B
:10B1900092E616246B00FB18059306ABE418059B9A
:10B1A00021001889FCF730FD011E03D1059B012405
:10B1B0001E8973E77888924B2288069C0993430086
:10B1C0001B5B904E013BDBB2029300230096019380
:10B1D000099BFFF71BFD041E02D0059B1E895DE73E
:10B1E0007B88069A5B009B5A079A1088328812184F
:10B1F000934202DC1B1A013B33807F4C02303288C1
:10B200000999001900F04CFC2388328801359B18FD
:10B210002380EDB2A8E70BAA3B7B7989388900929D
:10B220003A000D32FCF708FC00250590059B002B29
:10B2300004D10A24002D00D16EE060E0059B7888DF
:10B24000197AFCF7C3FB0100041E63D1694C6C4BF7
:10B25000788806940993069B4400E45A694B063C9F
:10B26000E4B20BAE328807930294019100930599E2
:10B27000099BFFF7CBFC041E4CD1079B5E491B8842
:10B280001A1D002D30D14A80059B5B4C5A896319E9
:10B290001A716B1C9BB2E318120A1A71162306A8C6
:10B2A00032881B1879890598FCF722FDFF21AA1C1A
:10B2B0002E1D03350B00059092B2B6B2ADB2002838
:10B2C00003D006ABDB8AD9B21B0AA218651911712B
:10B2D0002B714C4D301D2A884949201800F0E0FBA5
:10B2E0002B88F618B5B2A1E74988914207D17A8830
:10B2F00006995200525AEB18053A9A42C4DC3E4C69
:10B300002800618800F0FCFB207021007888FAF7A3
:10B310005FFED1E5002DF2D13E89BFE6162606ABD1
:10B32000F61831003889FCF76FFC3D000400FA354F
:10B3300000282DD0037A9B060CD400227B89398902
:10B34000788800923A000C32FFF7E8FB041E10D018
:10B350003E8915E03088FFF741FB00281AD083684A
:10B36000002B17D02100122278889847041EE4D0C1
:10B37000EEE72B78002B02D17888FAF739FE002609
:10B380002B78002B00D097E5002C00D194E585E6C2
:10B390000124DDE70E24DBE7162506ABED182900B6
:10B3A0003889FCF731FC041E47D0037A9B0611D480
:10B3B000154A7B881188994203D01448814207D1ED
:10B3C0001380134BF2261D780023D9B2A94221D352
:10B3D0000924A1E72888FFF701FB00282FD0836804
:10B3E000002B2CD02100122278889847041EDFD031
:10B3F00092E7C0465864FF1F2868FF1F2A68FF1F96
:10B400001C69FF1F0C6AFF1F086BFF1FFFFF000076
:10B41000066BFF1F31005943546801336018615AAD
:10B420000029D2D13C0008342100F22200F038FB80
:10B4300021007888FAF7E4FD3EE501246CE70E244C
:10B440006AE71D4B1A887B889A4231D07888FAF7D0
:10B45000E1FD31E5F223059851684343CD18C95AFF
:10B4600000291FD03B7A012B0BD16C88AB887888E0
:10B47000AA1D0094FFF752FB041E02D000233B726A
:10B480002E88F2220021280000F0C2F900232B8030
:10B49000059B0133DBB20593084B05991B78064ADF
:10B4A0008B42D7D801235B421380002CCED0F5E528
:10B4B000002634000596EFE7086BFF1F066BFF1FA1
:10B4C00070B504000E001500FFF796FA031E08D1B0
:10B4D00031000548FFF790FA03001120002B02D03D
:10B4E0001C8000209D7070BDFFFF0000F8B50B4F61
:10B4F00006003B780D001400FF2B0ED00A2000F050
:10B5000037FA011E09D0B12303800023468003715E
:10B51000C5800481387800F0EBF8F8BD3544FF1F92
:10B52000F7B50F0008A90600088809A90B240988A7
:10B53000002821D10234022B1ED1557813782D0218
:10B540001D432B008B4301937334002B14D1FB68F4
:10B55000300019000093FFF74FFB019C85420BD090
:10B560002A0030000099FFF7ABFF041E04D12A0027
:10B5700030007989FFF7BAFF2000FEBDF0B50E78E4
:10B5800085B003900AA805880120022E0DD14C68D1
:10B590002778647824023C43054FBC4205D10398C8
:10B5A000DBB201960095FFF7BBFF05B0F0BDC046CA
:10B5B00002290000034B10B51B68002B00D09847F0
:10B5C000FEE7C046146BFF1F07B501A8FFF7F2FFA7
:10B5D000044A05480021121A00F04AF9F8F70AF95E
:10B5E000FEE7C046186BFF1F3844FF1F0000000035
:10B5F00001B40248844601BC604700BF51470100C6
:10B6000001B40248844601BC604700BF311B000002
:10B6100001B40248844601BC604700BF193BFF1FCC
:10B6200001B40248844601BC604700BF193AFF1FBD
:10B6300001B40248844601BC604700BFC51D00003C
:10B6400001B40248844601BC604700BF4551010077
:10B6500001B40248844601BC604700BF1D4B010095
:10B6600001B40248844601BC604700BF8538FF1F13
:10B6700001B40248844601BC604700BF456B01002D
:10B6800001B40248844601BC604700BF350E00008B
:10B6900001B40248844601BC604700BFC52DFF1FAE
:10B6A00001B40248844601BC604700BF090E000097
:10B6B00001B40248844601BC604700BF791800000D
:10B6C00001B40248844601BC604700BF792DFF1FCA
:10B6D00001B40248844601BC604700BF691F0000F6
:10B6E00001B40248844601BC604700BF55490100CF
:10B6F00001B40248844601BC604700BF594F0100B5
:10B7000001B40248844601BC604700BFC521000067
:10B7100001B40248844601BC604700BF014C0100EF
:10B7200001B40248844601BC604700BF6571010056
:10B7300001B40248844601BC604700BF6DBC0000F4
:10B7400001B40248844601BC604700BF8D1200006E
:10B7500001B40248844601BC604700BF0132FF1FAC
:10B7600001B40248844601BC604700BFF54E0100A9
:10B7700001B40248844601BC604700BFD92FFF1FB7
:10B7800001B40248844601BC604700BFC94A0100B9
:10B7900001B40248844601BC604700BF091B000099
:10B7A00001B40248844601BC604700BF350E00006A
:10B7B00001B40248844601BC604700BF4D38FF1FFA
:10B7C00001B40248844601BC604700BF5D17000019
:10B7D00001B40248844601BC604700BFA54F010088
:10B7E00001B40248844601BC604700BF1147010014
:10B7F00001B40248844601BC604700BF59520100B1
:10B8000001B40248844601BC604700BF6130FF1F9D
:10B8100001B40248844601BC604700BF154D0100D9
:10B8200001B40248844601BC604700BFC9A90000BA
:10B8300001B40248844601BC604700BFD91AFF1F0B
:10B8400001B40248844601BC604700BF4537FF1F72
:10B8500001B40248844601BC604700BFC92600000D
:10B8600001B40248844601BC604700BFC538FF1FD1
:10B8700001B40248844601BC604700BFB70E000017
:10B8800001B40248844601BC604700BF1930FF1F65
:10B8900001B40248844601BC604700BF055E000059
:10B8A00001B40248844601BC604700BFA9460100BC
:10B8B00001B40248844601BC604700BF75A900007E
:10B8C00001B40248844601BC604700BF2526000041
:10B8D00001B40248844601BC604700BFD91B000088
:10B8E00001B40248844601BC604700BF2146010004
:10B8F00001B40248844601BC604700BF5933FF1FB2
:10B9000001B40248844601BC604700BF9135FF1F67
:10B9100001B40248844601BC604700BFC56D010008
:10B9200001B40248844601BC604700BFADAE0000D0
:10B9300001B40248844601BC604700BF3D180000C6
:10B9400001B40248844601BC604700BFB14E00000C
:10B9500001B40248844601BC604700BFE117000003
:10B9600001B40248844601BC604700BF3D4B010062
:10B9700001B40248844601BC604700BF1D4D010070
:10B9800001B40248844601BC604700BF2951010050
:10B9900001B40248844601BC604700BF9D35FF1FCB
:10B9A00001B40248844601BC604700BFE54800007E
:10B9B00001B40248844601BC604700BF7139FF1FD3
:10B9C00001B40248844601BC604700BFB54C010089
:10B9D00001B40248844601BC604700BFE92800006A
:10B9E00001B40248844601BC604700BFED4A010033
:10B9F00001B40248844601BC604700BFF94C010015
:10BA000001B40248844601BC604700BF51250000D4
:10BA100001B40248844601BC604700BF434D0100A9
:10BA200001B40248844601BC604700BF2D3BFF1FA4
:10BA300001B40248844601BC604700BFF30E000019
:10BA400001B40248844601BC604700BF2932FF1F91
:10BA500001B40248844601BC604700BF0D5201009A
:10BA600001B40248844601BC604700BFDD520100BA
:10BA700001B40248844601BC604700BF5118FF1F53
:10BA800001B40248844601BC604700BF851F000026
:10BA900001B40248844601BC604700BF4D1F00004E
:10BAA00001B40248844601BC604700BFE94C010074
:10BAB00001B40248844601BC604700BF85520100C2
:10BAC00001B40248844601BC604700BF45500000F5
:10BAD00001B40248844601BC604700BF7D18FF1FC7
:10BAE00001B40248844601BC604700BF291C000025
:10BAF00001B40248844601BC604700BF810E0000CB
:10BB000001B40248844601BC604700BF090E000032
:10BB100001B40248844601BC604700BFC12FFF1F2B
:10BB200001B40248844601BC604700BF9DA90000E3
:10BB300001B40248844601BC604700BF413BFF1F7F
:10BB400001B40248844601BC604700BFB352010003
:10BB500001B40248844601BC604700BF01240000D4
:10BB600001B40248844601BC604700BFEDA5000057
:10BB700001B40248844601BC604700BF156B010058
:10BB800001B40248844601BC604700BFCD4C0100AF
:10BB900001B40248844601BC604700BFD949010096
:10BBA00001B40248844601BC604700BF2124000064
:10BBB00001B40248844601BC604700BF355500000F
:10BBC00001B40248844601BC604700BFDD66010045
:10BBD00001B40248844601BC604700BF8B5201009B
:10BBE00001B40248844601BC604700BFED39FF1F25
:10BBF00001B40248844601BC604700BF9136FF1F74
:10BC000001B40248844601BC604700BFC135FF1F34
:10BC100001B40248844601BC604700BF55220000C1
:10BC200001B40248844601BC604700BF0539FF1FCC
:10BC300001B40248844601BC604700BF3938FF1F89
:10BC400001B40248844601BC604700BF017F000088
:10BC500001B40248844601BC604700BF056A000089
:10BC600000010103020003030403050206020702A8
:10BC7000080209020A030B030C020D000E030F0356
:10BC8000100311001300140315001600C53B00112A
:10BC9000F93B00110000000002000000A2BC0011EE
:10BCA000192A0F180A000000F1590000FD240000B5
:10BCB000414601004580001159A00011AD740011EA
:10BCC000497E0011115300114DAE0011794F001142
:10BCD000B93D0011E93E00110000000016160000F9
:10BCE00002000000ECBC0011F4FFF3FFD2FC0000E6
:10BCF0002940001100000000000000005475796127
:10BD00000042312E34003030313900676974687573
:10BD1000622E636F6D2F707676780054483035460A
:10BD2000000000000200000038BD0011292A282A66
:10BD3000272A262A252A242A0A180000E2040000BD
:10BD40007102000078EC0000744000001027000031
:10BD500060F0000006640000204E000000000000BB
:10BD6000050000001F501D00023CB4000001190036
:10BD700014000000A1020000303132333435363770
:10BD80003839414243444546000000001557001130
:10BD9000695700110000000002000000A4BD00115E
:10BDA0006F2A6E2A1A18EAD8BC80F0FC60000000E6
:10BDB00000000000000000F505D39727B6F615F740
:10BDC000B777E6F0C7F27200000001A000000000A3
:10BDD0006410B71DC8206E3BAC30D9269041DC768C
:10BDE000F4516B6B5861B24D3C7105502083B8ED36
:10BDF00044930FF0E8A3D6D68CB361CBB0C2649B5A
:10BE0000D4D2D38678E20AA01CF2BDBDFB349B5F7E
:10BE1000800000800010000000000000AF600011F2
:10BE200039770011D3600011417B00115761001177
:10BE3000177B0011CD610011ED7A00111F62001116
:10BE4000B57C001187620011B57C0011B962001148
:10BE50006F7C0011CD610011A57A001145620011BF
:10BE60004D7C001100000000000000002B63001159
:10BE70004D7C00118D63001151770011052A042AB1
:10BE8000012A002A02290328012800280118001885
:10BE9000000000000000000000000000000000871B
:10BEA0000101020102010102010203030401030175
:10BEB000010101010303020103000D000E00100047
:10BEC000110013001401070108010A010B011C01F4
:10BED0001D02040205020702080219021A021C02CE
:10BEE0001D030103020317000201000504000807F7
:10BEF000000B0A001716001D1C01020101050401B8
:10BF00000E0D011110011413011716011A19020266
:10BF100001020B0A020E0D02111002141302171671
:10BF2000030504030807030B0A030E0D00010203B7
:10BF300007090A0B0E0F101112141718191A1B1FDC
:10BF40002021220095A7001151A800110000000037
:10BF5000020000008EBE0011000000007DB500113F
:0CBF600000000000020000008CBE001178
:020000041FFFDC
:1000000000000000213D0011A8BC0011A4BC00119B
:100010004461FF1F0000000000000000000000001D
:1000200000000000000000000000000000000000D0
:1000300000000000000000000000000000000000C0
:1000400000000000000000000000000000000000B0
:1000500000000000000000000000000000000000A0
:100060000000000000000000000000000000000090
:100070000000000000000000000000000000000080
:100080000000000000000000000000000000000070
:100090000000000000000000000000000000000060
:1000A0000000000000000000000000000000000050
:1000B0000000000000000000000000000000000040
:1000C0000000000000000000000000000000000030
:1000D0000000000000000000000000000000000020
:1000E0000000000000000000000000000000000010
:1000F0000000000000000000000000000000000000
:1001000000000000000000000000000000000000EF
:1001100000000000000000000000000000000000DF
:1001200000000000000000000000000000000000CF
:1001300000000000000000000000000000000000BF
:1001400000000000000000000000000000000000AF
:10015000000000000000000000000000000000009F
:10016000000000000000000000000000000000008F
:10017000000000000000000000000000000000007F
:10018000000000000000000000000000000000006F
:100190004D32FF1FAD30FF1FC1660100000000009F
:1001A000000000000000000000000000000000004F
:1001B000000000000000000000000000000000003F
:1001C000000000000000000000000000000000002F
:1001D000000000000000000000000000000000001F
:1001E000000000000000000000000000000000000F
:1001F00000000000000000000000000000000000FF
:1002000000000000000000000000000000000000EE
:1002100000000000000000000000000000000000DE
:1002200000000000000000000000000000000000CE
:1002300000000000000000000000000000000000BE
:1002400000000000000000000000000000000000AE
:10025000000000000000000000000000000000009E
:10026000000000000000000000000000000000008E
:10027000000000000000000000000000000000007E
:10028000000000000000000000000000000000006E
:10029000000000000000000000000000000000005E
:1002A000000000000000000000000000000000004E
:1002B000000000000000000000000000000000003E
:1002C000000000000000000000000000000000002E
:1002D000000000000000000000000000000000001E
:1002E000000000000000000000000000000000000E
:1002F00000000000000000000000000000000000FE
:1003000000000000000000000000000000000000ED
:1003100000000000000000000000000000000000DD
:1003200000000000000000000000000000000000CD
:1003300000000000000000000000000000000000BD
:1003400000000000000000000000000000000000AD
:10035000000000000000000000000000000000009D
:10036000000000000000000000000000000000008D
:10037000C9B50011000000000000000000000000EE
:10038000000000000000000000000000000000006D
:10039000000000000000000000000000000000005D
:1003A000000000000000000000000000591AFF1FBC
:1003B000000000000000000000000000000000003D
:1003C000000000000000000000000000000000002D
:1003D000000000000000000000000000000000001D
:1003E000000000000000000000000000000000000D
:1003F00000000000000000000000000000000000FD
:08183800206FFF1F4118FF1F84
:10184000024981F3088802F06FFA0000206FFF1F41
:1018500010B502F089FA072804D0122808D002280F
:1018600008D010BD044A0420136B01331363F8E75A
:101870000220F6E71420F4E70065FF1FF8B5070023
:101880000C0026002500503630785135002804D150
:101890000300287058342370F8BD2978CA00481E08
:1018A0008141A3183800A25C5B68C9B2FFF7D0FF82
:1018B00000280DD12B78DA00A218013350602B706C
:1018C0003378044A013B3370136A01331362D8E75B
:1018D0000123DFE70065FF1F5C234343074910B581
:1018E000C9180B0058331B78012B05D1FFF7C6FF31
:1018F000034A936A0133936210BDC0463465FF1FEB
:101900000065FF1F10B502F037FB064A01211300E6
:1019100010CB4942D967044B136002F0E5F920006F
:1019200010BDC04600E100E01000100010B504003A
:1019300002F022FB024B1C6002F0D6F910BDC0463B
:1019400000E100E0431E5A425341A022F0B5D2010B
:101950005B421340154D164A40019B182A18127E0F
:101960008BB00191002A1BD01A000832D46F0022DC
:10197000E6B206AFE4B294420EDC2818C369002B2D
:1019800008D0019902AA117106AA049202AA16733C
:1019900003A898470BB0F0BD1978B9540132EAE7B3
:1019A0001A7D1A7806AB01261A70E6E7C067FF1F9A
:1019B00000400040F0B5254B04004001C25C85B0FA
:1019C000002A2BD01A18117E002927D0917E0029D9
:1019D00024D01179022921D11689D788D168F51B25
:1019E000ADB22A1C102D00D9102292B2BE4217D1DE
:1019F0001818012303710023C269C38003819A422E
:101A000006D06846032103730171029301A8904731
:101A10000820002C00D0192001F0FEFA05B0F0BD1E
:101A2000013C65426C41A0256442ED012C40084D0B
:101A30001B186419074D0633013A92B2AA42EDD041
:101A40001888461C1E80085C2070F5E7C067FF1FE1
:101A500000400040FFFF00000F220E4B10B59868B9
:101A6000104002380A280BD802F060F80D0A0B0A61
:101A70000A110A0A0A0A060002210020FFF762FF83
:101A800010BD0121F9E70020FFF794FFF8E7DB6FB5
:101A9000F6E7C046004000400F220E4B10B5986894
:101AA000104002380A280BD802F040F80E0A0B0A40
:101AB0000A120A0A0A0A060002210120FFF742FF61
:101AC00010BD01210800F9E70120FFF773FFF7E7D8
:101AD000DB6FF5E70090004013B5334C2378072BFC
:101AE0003DD8324B1A78324B002A39D180221968FE
:101AF00052020A431A60252001F0C4FE20232D4A19
:101B000011680B43802113606B460422C9050868E5
:101B10000733104228D080210422C905C86810422A
:101B20002ED080212020C905CA688243CA601422B1
:101B30001A701A78002A2FD18021C905C86820326E
:101B40000243CA6014221A701A78002A28D11A4B4C
:101B50001A7D22785A601D221A705932DA6013BD3C
:101B60001A6816490A40C5E7086802430A60142249
:101B70001A701A78002ACED01A78013AD2B2F7E752
:101B8000C8680243CA6014221A7019784A1ED2B279
:101B90001A700029F9D1C4E71A78013AD2B2C7E71E
:101BA0001A78013AD2B2CEE77043FF1F3844FF1FC4
:101BB0003CF000406843FF1F00200040FFFFFEFF95
:101BC000564B70B51B68012B03D1554A936D0133F9
:101BD000936502F011F9534B534A1860534B544C20
:101BE0001A600123534A1360534A13602378002B71
:101BF00006D006225149524802F0A6F8002323706D
:101C0000504A514B10681B78C1B2002B0ED14F4C7B
:101C1000C0B223785BB2002B4FDB237824785BB211
:101C200064B21B0424021B191B1813600B1C5029DF
:101C30004ED95023464A47491078DBB2FF2202288A
:101C40004BD10868444C454D267890432A789642FB
:101C500054D9227824782E78023B5D10A31B6B4365
:101C60005201D31A10335B111843086002F054F983
:101C7000031F012B45D83A4B1B78002B06D0394B5C
:101C80001B78002B02D0002002F05EF9A122364B17
:101C900092009978354B4A431B689B188322920027
:101CA0009B181B78033B012B03D8AF20400001F0A9
:101CB00093FF01222E4BDA8270BD237824785BB229
:101CC00064B2FF33FF341B0424021B190138ABE755
:101CD000CAB2022AAED20223ACE70868254C264DD0
:101CE000267890432A78964208D9227824782D784D
:101CF000023B5B10641B63435201B2E72378DBB203
:101D0000B2E70228D5D11D4B1B78013B022B03D92A
:101D10001B4B1B78022BCCD16C20C8E79809FF1F06
:101D2000FC0FFF1F3864FF1FFF3F0000141003402B
:101D30003C64FF1F0C10034000100340D50BFF1F35
:101D40007211FF1FB40003408C09FF1F680AFF1FB8
:101D5000490AFF1F94000340460AFF1F470AFF1F5E
:101D6000F908FF1F2209FF1F300DFF1F3409FF1F55
:101D7000BC0BFF1F440AFF1F450AFF1F1C09FF1F62
:101D80002309FF1F10B502F0B7F80022014B1A809B
:101D900010BDC0463664FF1F10B502F055F8A121F2
:101DA000054A89009478054A61431268044B521829
:101DB000528C1A8010BDC046300DFF1F3409FF1F22
:101DC0003664FF1F10B50D4B0D4A9978A1239B0077
:101DD0004B431268D218531DD97F0A4B1B88994276
:101DE00009D2441C07D0C82805D0D2695B1A5A43CF
:101DF000054B5343C01801F0E7FF10BD300DFF1F26
:101E00003409FF1F3664FF1F7102000070B5244DB6
:101E10002B68002B28D001F017FF2B68D8402B68C7
:101E20000400002B27D002F0B7F82B68D8401D4BD8
:101E30001D4A9978A1239B004B431268D118D25CAC
:101E400091239B00002A20D0CA580132CA50174B58
:101E500017491B680868834214D3D23B181A012A19
:101E60001AD0144B186070BD01F0EEFE124B1968C9
:101E700001F082FED3E702F08FF80F4B196801F0F2
:101E80007BFED4E70D495B18E8E7CA500C4B1B6892
:101E9000DB68E418201AE4E7F530FF30E1E7C046DC
:101EA0001C08FF1F300DFF1F3409FF1F9C09FF1F77
:101EB0003864FF1FA009FF1F1808FF1F2DFF3F00F8
:101EC0004064FF1F70B504000D00282916D10300DF
:101ED000A433C2881B889B1A0B4A9BB293420DD92C
:101EE00006006A3605223100653001F0F5FF002852
:101EF00004D13100200002F01FF870BD290020003D
:101F000001F00AFFF9E7C046FE7F0000F8B50500C2
:101F1000012001F0B1FF134CA36AA26A9342FBD1E6
:101F2000114E336001F038FE10490300086010487C
:101F3000426894460F4A17680022BC4501D24268A5
:101F4000BA1A0D4802603268AD18A422E562606AD0
:101F5000520302436262094A1278002A01D00F3B01
:101F60000B60F8BD00F00040340AFF1FE408FF1FBB
:101F700028100040180AFF1F1C0AFF1F1C09FF1F22
:101F800070B580241025E405A3682B43A36001F0FD
:101F90000BFEA368AB43A36070BD0000F7B516004D
:101FA00080221C001023D2050191916805000B438B
:101FB000936000225A4BD7301A6001F055FE9D23E2
:101FC0002A002F009B00EB58CA3201210092FC37F7
:101FD000002B01D00021009A386801F0D5FE2900BD
:101FE000009BCB311A784F4BD3351A604B780A7867
:101FF0001B0213438A7812041A43CB781B0613433F
:10200000494A1BBA13604B790A791B0213438A7938
:1020100012041A43CB7931001B061343434A1BBAFF
:1020200013606B782A781B021343AA7812041A43B0
:10203000EB781B0613433E4A1BBA1360019A330226
:1020400013433C4A13603C4B22001B1B9C46032954
:102050003DDCB3089A0013005142B21A032A46D15C
:10206000354AE018511A827840781204000202437F
:10207000E05C043302430A600022FF2B4BDDF022B8
:102080002E4B12011A600F222D4B1A602D4A136835
:10209000002BFCD00023224A27491360091B321D64
:1020A0000B191B68043A180A23706070180C1B0E79
:1020B000A070E3700434002AF2DC802210213B6817
:1020C000D20501333B6093688B439360F7BD634651
:1020D000D578981893782D061B042B43157804396E
:1020E0002B43557804322D022B430360AFE7022ABD
:1020F0000AD1114AE05C511AE218527812020243E6
:102100000A6004339BB2B7E7012AB5D10A4A521AD2
:10211000E15C1160F5E7084959180A600433ACE73F
:10212000000004403C0004403800044034000440F7
:10213000300004400C00044000010440040004404E
:102140001000044014000440F7B5150080221C0064
:102150001023D2050091916807000B439360002380
:10216000654AD730136001F07FFD9D233E009B0040
:10217000F9583B00CA363200FC33002900D07FE01A
:10218000586801F001FE390032785C4BCB311A609F
:102190004B780A781B0213438A78AC4612041A4320
:1021A000CB78281D1B061343554A1BBA13604B7985
:1021B0000A791B0213438A7912041A43CB791B064E
:1021C0001343504A1BBA13604B7A0A7A1B0213431B
:1021D0008A7A12041A43CB7A21001B0613434A4A17
:1021E0001BBA1360009A2B021343484A1360220063
:1021F000474B1B1B0093009BCE785B1801938B7899
:1022000036061B0433430E78043833434E780431CA
:1022100036023343019E33600328ECDC0321A80817
:10222000431C9B002940800003292BD13849E51825
:102230005E18A9786D78E35C09042D0229431943DF
:102240003160030008330021FF2B2DDD314B324973
:1022500019600F21314B1960012327490B60304B66
:1022600019680029FCD006211B680B40042B20D0E4
:1022700080220020D20593680A318B439360FEBD13
:1022800001217DE7022908D121495D18E11849782B
:10229000E35C090219432960D3E70129D3D11C4922
:1022A0005918E35C0B60CCE7194818180160043337
:1022B000CAE7002310490B606346002B0CDC3B008F
:1022C000FC335A68102101325A608022D20593688B
:1022D00001208B439360D2E7009B9B181B68190A6F
:1022E00013705170190C1B0ED37004235B42917054
:1022F0009C440432E0E7C046000004403C00044037
:102300003800044034000440300004400C00044015
:102310000001044004000440080F000010000440C5
:102320001400044070B5061E19D002225A4B9B7946
:102330009343012B13D1594B1A78FF2A0FD15A78A6
:10234000FF2A0CD19A78FF2A09D1DA78FF2A06D120
:102350001A79FF2A03D15B79FF2B00D199E0504B0A
:102360000C201A78012A08D000224E4D1A702978C4
:102370000B00093B042B01D8212070BD4B1F012B02
:10238000FAD9454CA37B042B00D982E0A279032A19
:1023900000D97EE09A1ED2B2012A02D860881F2896
:1023A00077D9002E56D0012E73D1A0880128E3D012
:1023B000002907D1581E032803D801F0B7FB1217D4
:1023C00015122E702978481E032811D80025364B87
:1023D0001D602823237501F0A7FDA84227D0A58002
:1023E000CAE702212970EDE70421FBE70321F9E7A1
:1023F00007390129C0D82D490968C96A8906BBD5A2
:102400002B4908780028B7D1012A01D9002BB3D174
:1024100002230B708021274D2633890128782375EC
:1024200001F0A2FD80212878890101F0F5FC01234B
:10243000A380214B1B78002B0AD0FA2280211F4B4E
:1024400092001B8809025A431A4B187801F084FD48
:10245000002092E701F090FD2B78A680073B012B2E
:1024600003D917482E7001F0FFFC114B114C1A785C
:10247000002A06D080210022207889011A7001F0FC
:1024800073FD01F031FC80212078090201F06CFD20
:10249000DEE7122071E7C046A60BFF1F6B09FF1F86
:1024A0001A09FF1F1C09FF1F4809FF1F4064FF1F77
:1024B0002309FF1F1B09FF1F2109FF1F2C09FF1FF5
:1024C0000010004010B5002901D001F0F5FC10BD4E
:1024D000F7B5604B01919978A1239B004B435E4A6D
:1024E000060014681022E418D6235B00E058362357
:1024F000FF33E35C00279343222B41D1574B0F3A24
:102500001A600760012501F0FFFC019B1880E82399
:102510005B00E35C002B01D0B34258DD0023504F39
:10252000FB70AD33FF33E3581A68002A03D09B8851
:10253000DB439B071DD03823FF33E35C002B18D00F
:102540009B235B00E35C002B13D1D133FF33E35CAF
:10255000B3420EDAA4235B00E15AE018090A023103
:1025600001F0C2FC23000122FE33013E01351A872F
:10257000FA70E8235B00E35C002B2AD0A8B2FEBD12
:1025800003683D00002BBED081880430090A023167
:1025900001F0AAFCD6235B00E3581F60B2E72300DA
:1025A000B133BA00FF339858013781880430090AE3
:1025B000023101F099FCE8235B00E35CBB42EEDCF6
:1025C000E822F61AED1800235200A354A6E70027CC
:1025D000F1E7200001F030FB00281FD0002E1DDDA8
:1025E0007319882647190193B600200001F0FCFA00
:1025F0005A30800020184068013581880430090A6B
:10260000023101F071FC200001F0A6FBA359013357
:10261000A351BD4202D0019B9D42E6D1114BE35C28
:10262000002BABD095239B00E35C002BA6D00E4B78
:10263000E15A0029A2D00D4AA35C994202D9013384
:10264000A3549BE700231A212000A35401F0ACFB04
:1026500094E7C046300DFF1F3409FF1F00140340EC
:10266000E010FF1F5A020000720200005E0200002C
:102670000D4970B54A6E0D4CD2038B69D20BA24244
:1026800006D80B4D0224AA4204D901F0E5FA70BD28
:1026900002246442E21815007E2425402242F4D030
:1026A000A3432B438B61F0E700F000400A200000B9
:1026B000FC1C0000F8B51D4B1D4F1A78002A10D1E4
:1026C000BA7B002A02D101321A7003E0032AFAD041
:1026D000022AF8D001F028FC00220120154B1A70C4
:1026E000F8BD154B154D1C68154B9E7801232B70BA
:1026F0002878C0B200F0A2FBBB7B002B0BD101F00D
:102700005BFAA1239B007343E41883239B00E41826
:1027100023782B70E4E7032B02D101F09DFBF0E757
:102720000020022BDCD101F02FFCEAE71C09FF1F7F
:10273000A60BFF1F2309FF1F3409FF1F490AFF1FB4
:10274000300DFF1FF0B587B00EAD2F780FAD2D788F
:102750000593AC46634614000E4D0CAA12782E78F1
:1027600003930D9B009201932200059B029701F0B9
:102770004BFC2E70012C01D0042C08D1802206497C
:102780008B889343054A1278D20113438B8007B09C
:10279000F0BDC0461C09FF1F6C11FF1F7809FF1F09
:1027A0000B001B3B70B504003020E02B0DD813004C
:1027B000E025493BFF3B9BB2ED00AB4205D8034B04
:1027C000200019825A8201F057FA70BD8410FF1F51
:1027D00010B501F011FB054B00205B68052B04D9F7
:1027E000034A5268D20200D4980810BD001000407D
:1027F000FCE100E070B501F0BFFB0D4B1B68FC3342
:10280000DC691D6AFFF7E4FF6419844204D2094BB6
:1028100001241B68002B07D004220024064B1A70E9
:10282000064A93690133936101F05EFA200070BD9E
:102830004064FF1F9809FF1F2309FF1FFC0FFF1FA4
:1028400070B50C4D2B68FC335C6A01F095FBFFF70B
:10285000BFFF2B680025FC339B6AE318834204D238
:10286000054B1B68AB4200D1051B01F03DFA280067
:1028700070BDC0464064FF1F9809FF1FD722044B5C
:1028800092009B5810B5002B00D0984710BDC04651
:102890000000FF1F10B501F0D3F8FFF7EFFF274945
:1028A000274BCA6D274C1A4084235B001343CB652A
:1028B000254B1B68186A01F0DFFA244B244A1A6082
:1028C000244B254A1A60A022244B52001A60244B44
:1028D000187801F051FA2000224901F09DFB0023F5
:1028E000A3600233A360204B2049236003232048C8
:1028F000A36001F091FB10221E4BFF201A60802282
:1029000052031A60802292031A60802212041A6015
:1029100001F01AFB012001F03FFAFA20400001F01B
:1029200063FA582001F058F9134801F045FA0120E4
:1029300001F072F9072001F04FFA10BD00F00040DD
:1029400000FEFEFF141000404064FF1F0000034023
:102950000180063DBC00034034080000A400034091
:102960004A0AFF1F71020000C3090000FFFF3F0079
:102970002810004000E100E030750000674E336829
:1029800088331B6883F3088801F0E6F8644A6549D8
:10299000136800200B401360634B644A1B6893422A
:1029A00000D1A6E001F070FA0221614A13688B435E
:1029B0001360FFF76FFF5F4B5F4C1878C0B201F0F8
:1029C00073FA0023A3600233A3605C4B01202360F1
:1029D00001F052FA0323A36001F016FA040001F09B
:1029E0000BFA050001F010FA554B186001F0E4FAFB
:1029F000544B1968621A531EA14200D21300802260
:102A0000D203934201D39B029B0A3268D16AC90761
:102A100000D471E04C491C0C09689BB24C435943EB
:102A20002402090A641803264849FC3293680A689C
:102A300047489B1A474A0768126847499B18474A04
:102A40009A1833409208DB190A600360042B03D9FB
:102A5000013233400A6003600E684149A619300014
:102A600001F08AF83F4F3E493B68C3183B60300095
:102A7000019301F011F93C4E306808183849306074
:102A8000884205D9019B01333B6001F005F93160B3
:102A900001F00AF9354B1B78002B0DD001F0ACF991
:102AA000334B621B196812188A4232D24919091B2A
:102AB000091A304801F0B0FA2F4E337A002B0ED0AD
:102AC00001F09AF9621BF1681218914224D9491950
:102AD000091B091A294801F09FFA00233372284B79
:102AE00083F3088801F090F8002001F0CDF901F09F
:102AF000ABFA01F0C9F95CE7DC0199000234641A11
:102B00005900641A09214B438033CB40A408E418D0
:102B100089E7FA218900CCE71A49DBE74064FF1F07
:102B20001CF00040FFFFC1FF0C0AFF1FB64121034C
:102B300010000040490AFF1F14100040C3090000A4
:102B4000100AFF1F340AFF1F380AFF1F200AFF1F49
:102B5000280AFF1F1C0AFF1F240AFF1FC4090000C8
:102B6000710200006008FF1F2C0AFF1F1C09FF1FD5
:102B7000E408FF1F00100040740BFF1F3C100040D2
:102B800000000020DC050000A022054B92009B58AD
:102B900010B5002B01D0984710BD01F045F8FBE7B8
:102BA0000000FF1FA122054B92009B5810B5002B7F
:102BB00001D0984710BD01F037F8FBE70000FF1F78
:102BC000A222054B92009B5810B5002B01D09847CC
:102BD00010BD01F029F8FBE70000FF1FA322054B01
:102BE00092009B5810B5002B01D0984710BD01F002
:102BF0001BF8FBE70000FF1FA422054B92009B5827
:102C000010B5002B01D0984710BD01F00DF8FBE77F
:102C10000000FF1F70B501F0EFF84F4B186001F096
:102C2000E3F90400C30702D401F06EF870BD00227E
:102C30004A4B1A604A4B18780138042829D800F00A
:102C400075FF0320181C2400200001F0ADF90128B5
:102C5000ECD0444C2378042B6ED100F095FF002873
:102C6000E4D001F0E1F9582000F0B6FF0223237010
:102C7000DCE7200001F008F8E9E7200001F0ACF9FA
:102C8000E5E7200001F038F8E1E7200000F09CFFC4
:102C9000DDE701F041F90500012808D1324B1B782E
:102CA000053B012B03D82000FFF76EFFD1E72D4B2A
:102CB0001B78022B01D0052B20D1022D28D12B4BC4
:102CC0009B7BAB431CD12000FFF76CFF264B187891
:102CD0000128BED16405BCD4244925224B7B034284
:102CE00005D1233A13405A42534126331A000B7D33
:102CF0009342AED9322000F0EFFFAAE7022D07D1B0
:102D0000194B1B78052B11D12000FFF759FFDDE788
:102D1000012D0BD1012B03D12000FFF75FFF98E7B6
:102D2000062B03D12000FFF767FF92E7200000F099
:102D30007BFF022D8DD1C9E7032B04D10C4B987C6E
:102D400000F0BAFF72E7072B00D06FE7094B987BC2
:102D500000F0F2FF6AE7C0469C09FF1F9809FF1FB9
:102D60009009FF1F2309FF1F1C09FF1FA60BFF1F50
:102D7000BC0BFF1FD40BFF1FFA210A4B0A4A490064
:102D80001A640A4A5A500A4A04395A50094A083100
:102D90009A64094A5A50094A5C315A50084ADA661C
:102DA0007047C0460000FF1F4527FF1F4128FF1F37
:102DB000F527FF1F2523FF1FB526FF1FC51DFF1F7A
:102DC000991DFF1F10B500F099FE10BDF7B50B0C53
:102DD000FF270122009300233C001E001D009446A3
:102DE000019089B262469A40100008401841361896
:102DF000B6B2FF2F02D1012E00D19FB2009802403F
:102E00001A41AD18ADB2FF2C02D1012D00D19CB2F8
:102E10000133102BE6D10320012E07D1012D04D15F
:102E2000019B2401E4191C700138FEBD102EFCD159
:102E30000238102DF9D00230F7E700008023F7B5F3
:102E40009C46264B264F01932649274A274D284C5E
:102E5000284B02281AD1604638600868264E304058
:102E6000802636033043086001990978002909D18A
:102E70001660224A2A60224A2260E02219689143A1
:102E8000A03A1BE08021C9021160F2E766463E606D
:102E90000F68194E3E408027FF023E430E600199A5
:102EA000097800290DD1176001280ED1154A2A6032
:102EB000154A2260E02219689143C03A0A431A6019
:102EC000F7BD802189021160EEE7E0210F4A02433D
:102ED0002A600F4A22601A688A43F0E74B0AFF1FF4
:102EE000E0000340D800034090000340000003408E
:102EF0005000034040000340FFFFE3FF0280063D17
:102F0000804508220180063D8066082200800698E0
:102F100080550822F8B51E4B80261A680020140040
:102F20003440324232D11A681A4F32431A600122B9
:102F30003B68063093433B6000F09EFF0122164D34
:102F40002B681E432E603B680A2613433B60802794
:102F5000BF00124B1B683B4211D1013EF6B2FF2E5F
:102F600009D17E220E4B1C682B68E40B144093435E
:102F700023432B6005E0082000F07EFFE9E7002EE8
:102F8000EFD180222B68600893432B60F8BDC046C8
:102F9000C4F000405CF0004018F0004068F00040D1
:102FA00060F0004010B500F027FE01215820034AD0
:102FB00000F0DAFDFFF7AEFF10BDC046600AFF1F4C
:102FC00010B578220021034800F07EFE01F014F8CD
:102FD000002010BD4867FF1F70B5040000F0CCFF53
:102FE00000230C200B4A010059438D18515C002925
:102FF0000DD0A14208D1012300246B7000F064FFC2
:1030000000F072FE200070BD01330A2BEBD11224B8
:10301000F6E7C0464867FF1F70B5040000F0ACFF3C
:10302000002319001D000D4A1078002806D0A04288
:103030000CD1557001310C320A29F5D1002B0AD17F
:1030400000F0DAFF00F050FE002070BD5078461E00
:10305000B0411B18EEE700F037FFF3E74867FF1FAA
:10306000F7B504000C20002384460E4D01926746FC
:103070005F43E85D7E19A04212D000280BD10A4BB5
:103080009C4662461B7808331370019B70707C5518
:103090007160B360FEBD01330A2BE8D10320F9E76C
:1030A0000720F7E74867FF1F4467FF1F8020F8B538
:1030B000484BC0051B68C1248360474BFF251A6835
:1030C000012313434361454BA4001A68444B40213C
:1030D0001A60444B1A68444B1A60444B1A59AA436D
:1030E0001A51C52292009E58AE4331438026995012
:1030F0009F583F49F6010F403E439E509E588027FF
:103100003602360A3043985080201A5900020A408D
:1031100002431A5104341A59364E3F043240802675
:103120003A431A511A5936061202120A32431A51F8
:1031300008341A5980260A4002431A51C3229200C9
:103140009F58B446AF4337439F509F58294E0F4076
:1031500007439F509F5837408026360437438026C8
:103160009F509F5836063F023F0A37439F50C02268
:103170001F59AF433A431A511A591202120A164301
:10318000C6221E5192009C58AC4365462C439C506D
:103190009C5800250C4020439850C72080001A58A6
:1031A000154C1140C02212020A431A50134B1B78CF
:1031B000DB08AB4201DC0020F8BD2378002B06D0F1
:1031C000A368002B00D0984701350C34EEE712209D
:1031D000F2E7C0466C43FF1F6843FF1FB0F000409A
:1031E0004067FF1FB4F000403C67FF1F00E100E0B4
:1031F000FF00FFFFFFFF00FF4867FF1F4467FF1F3F
:10320000030010B51F2809D8072200201340072407
:1032100004490A78A24313430B7010BD0023062013
:10322000F5E7C0464467FF1F054B06491B780A684F
:1032300005485B0702401B0B134300200B607047DF
:103240004467FF1F1CF00040FFFFC1FF70B50C2555
:10325000FFF7EAFF0A4B1C780A4BE4086543ED18B8
:10326000002C01D1200070BD2B78002B06D06B689C
:10327000002B00D09847013C0C3DF1E71220F2E70B
:103280004467FF1F3C67FF1F1FB5002102220B0090
:1032900001910091052000F0CFFE02230B490A683E
:1032A0001A42FCD120230393039B5A1E0392002B46
:1032B000FAD1074A1368002BFCDA0B246C44200077
:1032C000012100F0B9FD207804B010BD90C8004085
:1032D00000C8004013B504000A4B0193019B002B6A
:1032E00001D1112016BDFFF7CFFF23000340044298
:1032F00005D0052000F0C0FD019B013BEDE7180063
:10330000F0E7C046FFFFFF0707B500F035FE80225B
:103310000821D205936A0191002B01D107399162EE
:1033200002210C4A11600199481E01900029FAD12E
:1033300003311160053101910199481E0190002966
:10334000FAD11160002B02D18022D205936200F0E5
:10335000CBFC07BD00C00040F0B52D4C89B02378F0
:10336000002B4FD1FEF7CEFA02232A4F03903A6882
:103370001A42FCD120230693069B5A1E0692002B6C
:10338000FAD1254E3368002BFCDA0120FFF7A2FFAB
:10339000011E02D0112009B0F0BD030003220190EC
:1033A000009005AD9F2000F047FE0321280000F0AB
:1033B00043FD02233A681A42FCD120230793079B5E
:1033C0005A1E0792002BFAD13368002BFCDA012039
:1033D000FFF780FF0028DDD10398FEF7A7FAAA784F
:1033E0006B7811041B020B4329780B4363601300B5
:1033F000113B0A49052B07D801239340A3600B60BA
:10340000012323700020C6E780231B03F6E7C04694
:103410005443FF1F90C8004000C800409808FF1F99
:103420001E4B30B55A6818781D4B85B0D3185942D9
:103430004B4101210093002300F0C6FD194B1A4AAD
:1034400002259A6300221A6510325A658022C4212F
:103450009D65164B1648D202DA6789004258154B13
:1034600080241A4080231B041343435064234120CB
:103470000393E40500F006FA402000F003FA6562C9
:10348000039D6B1E0393002DFAD103236362FFF7A4
:103490003BFFA562FFF760FF05B030BD6043FF1F33
:1034A00095FFFEF700C80040050001FF04E100E0C1
:1034B00000E100E0FFFF00FFF0B585B00700FEF778
:1034C00021FA022305002D4C22681A42FCD1202348
:1034D0000093009B5A1E0092002BFAD1284E3368AD
:1034E000002BFCDA0120FFF7F5FE002803D01124A1
:1034F000200005B0F0BD234B2360022322681A424E
:10350000FCD120230193019B5A1E0192002BFAD17A
:103510003368002BFCDA0120FFF7DCFE0028E6D13F
:10352000194B1F60022322681A42FCD12023029308
:10353000029B5A1E0292002BFAD13368002BFCDA50
:103540000120FFF7C7FE0028D1D1104B23600223D2
:1035500022681A42FCD120230393039B5A1E039234
:10356000002BFAD13368002BFCDA0120FFF7B2FE02
:10357000041EBCD12800FEF7D9F9B9E790C8004075
:1035800000C8004001000006A8C8004001800001FA
:1035900010B50020FFF790FF10BD000010B5064BDE
:1035A00018705960FFF73CFF00211320034AFFF712
:1035B00057FD002010BDC0466043FF1F2134FF1F90
:1035C000F0B5040085B003920291FEF79BF98822C2
:1035D00063035B0B52051A438023DB059D6A80233E
:1035E000274F0092BA68002601901B039A420CD91B
:1035F000F82326001B041E401C4206D08022214BCB
:1036000052025E6219680A431A60002D0BD100F065
:10361000B3FC02221C4B1A608023DB055A62013A7C
:103620009A6200F061FB0023039A934220D1002D9F
:103630000AD100F0A1FC144B03221D608023DB059E
:103640005A629D6200F050FB8023BA681B039A42C5
:1036500008D9002E06D000220A4B0C495A621A687B
:103660000A401A600198FEF761F9002005B0F0BD2C
:10367000009A0299D2181278CA540133D4E7C0468E
:103680005443FF1F00C8004000C00040FFFFFEFF82
:10369000F0B587B0029103920400FEF733F9019070
:1036A00000F06AFC802302250122234EDB053560F1
:1036B0005D629A6200F018FB204F3B682B42FCD100
:1036C00020230493049B5A1E0492002BFAD11C4D14
:1036D0002B68002BFCDA0120FFF7FCFD002802D04C
:1036E000112007B0F0BD2000039A029900F0D4FB2E
:1036F000022304003A681A42FCD120230593059B5B
:103700005A1E0592002BFAD12B68002BFCDA0120FF
:10371000FFF7E0FD051EE3D100F02EFC802303221D
:10372000DB0535605A629D6200F0DEFA0198FEF713
:10373000FDF8E0B2D5E7C04600C0004090C80040A8
:1037400000C80040F0B5802489B00600FEF7DAF822
:10375000E405A36A02250393029000F00DFC012307
:10376000304F3D606562A36200F0BEFA2E4C2368C4
:103770002B42FCD120230593059B5A1E0592002B5A
:10378000FAD12A4D2B68002BFCDA0120FFF7A2FDAD
:10379000002803D01124200009B0F0BD244B236081
:1037A000022322681A42FCD120230693069B5A1E4C
:1037B0000692002BFAD12B68002BFCDA0120FFF7D0
:1037C00089FD021EE6D11B4B03211E600300019000
:1037D0000090202000F030FC022322681A42FCD125
:1037E00020230793079B5A1E0792002BFAD12B68C0
:1037F000002BFCDA0320FFF76DFD041ECAD100F098
:10380000BBFB80230322DB053C605A629C6200F014
:103810006BFA039B002B01D1FFF776FD0298FEF7B0
:1038200085F8B8E700C0004090C8004000C80040DC
:103830000100000694C8004007B50002019104226F
:10384000000A01A9FFF724FF0EBD000073B50500B3
:1038500005240B4AA3005B429B1819686B46DE1DCA
:103860003000FFF7B3FA022804D133782B55013C1E
:10387000EFD276BD052CFCD00128FAD10230F8E752
:10388000140900111F2807D8012380228340D20584
:1038900091680B43936070473F2808D8012380222A
:1038A00020388340D20551690B435361F3E75F2809
:1038B000F1D80123802240388340D205116A0B439E
:1038C0001362E8E71F2807D8012280218240C9053A
:1038D0008B6893438B6070473F2808D80122802172
:1038E00020388240C9054B6993434B61F3E75F2859
:1038F000F1D80122802140388240C9050B6A9343E8
:103900000B62E8E71F2810D880230200DB05153A78
:103910001968012A06D820229143196019680A43C0
:103920001A60704701228240F6E73F2811D88023B1
:103930000200DB05353AD968032A06D810229143E4
:10394000D960D9680A43DA60EBE701222038824067
:10395000F5E75F28E5D842238022181A413B8340CF
:10396000D205516A99435162516A0B435362D8E7B9
:1039700010B50400012813D1A022184992050B6844
:103980005B015B0913430B60154B164A1968114024
:10399000154A0A431A60402219680A431A6010BD8A
:1039A0000028FCD101000A2000F056FB21000B206A
:1039B00000F052FBC0220A4B920019680A434021D2
:1039C0001A601A688A431A60B022044912060B680A
:1039D0005B015B0913430B60E1E7C04614F0004054
:1039E0001CF000407F00FEFF80FD010072B6074A18
:1039F0001368013313600422054B1A600023054A43
:103A000013608022D2055360FEE7C0467808FF1F8E
:103A1000C0F00040C4F0004005490B68002B05D100
:103A2000044A0A6004490A60044A13607047C046A9
:103A3000140AFF1F841E0000380AFF1FC4F0004054
:103A40000023034A1360034A1360034A136070475C
:103A500054F0004040F1004044F10040002310B514
:103A6000184C8AB0009301932378012B27D0694624
:103A7000012000F0D9F9002817D1009B12490293C8
:103A8000019B06AA0393114B02A81B680493104BD9
:103A90001B68059300F088F810220E4906A800F074
:103AA0001BFA002804D1FF23237000200AB010BDA8
:103AB0000123094A074902A8237000F075F8012084
:103AC000F4E7C0464464FF1F1029001108290011C3
:103AD0000C290011202900114864FF1F13B501248F
:103AE0006946012000F0A0F9034B00940193FFF711
:103AF000B5FF200016BDC046BB0B000010B5FFF798
:103B00009FFFFFF7EBFF002802D0024B984710BD44
:103B1000FEE7C046E1A2000002B471464908490030
:103B2000095649008E4402BC7047C04602B4714633
:103B300049084900095C49008E4402BC7047C046F0
:103B400003B47146490840004900095A49008E44AF
:103B500003BC70470000000001B40248844601BC69
:103B6000604700BFC9A9000001B40248844601BCF7
:103B7000604700BF0167010001B40248844601BCF0
:103B8000604700BF090E000001B40248844601BC32
:103B9000604700BF01D7000001B40248844601BC61
:103BA000604700BFBD5C010001B40248844601BC0F
:103BB000604700BFDD3F000001B40248844601BCFD
:103BC000604700BFE9F6000001B40248844601BC2A
:103BD000604700BFF935010001B40248844601BCCA
:103BE000604700BF7912010001B40248844601BC5D
:103BF000604700BFD9B0000001B40248844601BC50
:103C0000604700BFED68010001B40248844601BC72
:103C1000604700BF7997000001B40248844601BCA8
:103C2000604700BFE512010001B40248844601BCB0
:103C3000604700BFE917010001B40248844601BC97
:103C4000604700BF71B0000001B40248844601BC67
:103C5000604700BFE90B010001B40248844601BC83
:103C6000604700BFD1AE000001B40248844601BCE9
:103C7000604700BF8944000001B40248844601BC8B
:103C8000604700BF116E000001B40248844601BCC9
:103C9000604700BF0934010001B40248844601BCFA
:103CA000604700BF090E000001B40248844601BC11
:103CB000604700BFD544010001B40248844601BCFE
:103CC000604700BF4DF9000001B40248844601BCC2
:103CD000604700BFB70E000001B40248844601BC33
:103CE000604700BF6137010001B40248844601BC4F
:103CF000604700BF9DA9000001B40248844601BC92
:103D0000604700BFF535010001B40248844601BC9C
:103D1000604700BFDD0A010001B40248844601BCCF
:103D2000604700BF51B8000001B40248844601BC9E
:103D3000604700BFD1B5001101B40248844601BC00
:103D4000604700BFC1F7000001B40248844601BCCF
:103D5000604700BFE94C010001B40248844601BC41
:103D6000604700BF5976010001B40248844601BC97
:103D7000604700BFE927000001B40248844601BC47
:103D8000604700BFEDA5000001B40248844601BCB5
:103D9000604700BF2144000001B40248844601BCD2
:103DA000604700BF6911010001B40248844601BCAC
:103DB000604700BF53B9000001B40248844601BC0B
:103DC000604700BF8D11010001B40248844601BC68
:103DD000604700BF8937010001B40248844601BC36
:103DE000604700BFF90D010001B40248844601BCE0
:103DF000604700BF8512010001B40248844601BC3F
:103E0000604700BFC95C010001B40248844601BCA0
:103E1000604700BF156B010001B40248844601BC35
:103E2000604700BF0D52010001B40248844601BC46
:103E3000604700BFE1AC000001B40248844601BC09
:103E4000604700BF3D71010001B40248844601BCD7
:103E5000604700BFF9ED000001B40248844601BC90
:103E6000604700BF75F8000001B40248844601BCF9
:103E7000604700BFC1A5000001B40248844601BCF0
:103E8000604700BF0189000001B40248844601BCBC
:103E9000604700BF016C010001B40248844601BCC8
:103EA000604700BF9573010001B40248844601BC1D
:103EB000604700BF8914010001B40248844601BC78
:103EC000604700BFE9D4000001B40248844601BC49
:103ED000604700BF21A9000001B40248844601BC2C
:103EE000604700BFCD4C010001B40248844601BCCC
:103EF000604700BFC115010001B40248844601BCFF
:103F0000604700BF8D82000001B40248844601BCB6
:103F1000604700BFCD0C010001B40248844601BCDB
:103F2000604700BFDD0C010001B40248844601BCBB
:103F3000604700BFA9D8000001B40248844601BC14
:103F4000604700BF85C1000001B40248844601BC3F
:103F5000604700BFED6B010001B40248844601BC1C
:103F6000604700BF8B52010001B40248844601BC87
:103F7000604700BFB352010001B40248844601BC4F
:103F8000604700BF75A9000001B40248844601BC27
:103F9000604700BF19FA000001B40248844601BC22
:103FA000604700BF6D0B010001B40248844601BCAC
:103FB000604700BF0134010001B40248844601BCDF
:103FC000604700BFC166010001B40248844601BCDD
:103FD000604700BFC56D010001B40248844601BCC2
:103FE000604700BF0534010001B40248844601BCAB
:103FF000604700BFBD0B010001B40248844601BC0C
:10400000604700BFADAE000001B40248844601BC69
:10401000604700BF9D6A000001B40248844601BCAD
:10402000604700BF2D6C010001B40248844601BC0A
:10403000604700BF6DF6000001B40248844601BC31
:10404000604700BF496D010001B40248844601BCCD
:10405000604700BF8552010001B40248844601BC9C
:08406000604700BF29A2001116
:10406800020000008ABE00110100000098BC001187
:104078000200000086BE001101000000A840FF1FDA
:1040880002000000A0BC001101000000C461FF1F75
:104098000200000084BE0011030000003861FF1F09
:1040A80012000000020000008ABE0011010000009A
:1040B800E0BC00110200000086BE001101000000F3
:1040C800DDBC001102000000EABC00110300000082
:1040D8007361FF1F0200000084BE0011030000008E
:1040E8008861FF1F0200000086BE00110100000069
:1040F800DCBC001102000000E8BC00110300000055
:104108004961FF1F0200000084BE00110300000087
:104118006A61FF1F020000008ABE00110100000052
:1041280024BD00110200000086BE0011010000003D
:10413800F141FF1F0200000036BD00110100000020
:104148001BBD00110200000086BE00110100000026
:10415800F041FF1F0200000034BD00110100000003
:104168009061FF1F0200000086BE001101000000E0
:10417800EF41FF1F0200000032BD001101000000E6
:104188000BBD00110200000086BE001101000000F6
:10419800EE41FF1F0200000030BD001101000000C9
:1041A80006BD00110200000086BE001101000000DB
:1041B800ED41FF1F020000002EBD001101000000AC
:1041C80001BD00110200000086BE001101000000C0
:1041D800EC41FF1F020000002CBD0011010000008F
:1041E800FCBC0011020202020202000000000000F2
:1041F80016150000A14B0011674B001178BD001186
:1042080090011D0018001800FFFF070102030405B4
:104218000602010600000000000000000000000087
:104228000000000000000000000000000000000086
:1042380003000000020000008ABE00110100000017
:1042480098BD00110200000086BE001101000000A8
:10425800AC42FF1F02000000A2BD001101000000D7
:10426800BE61FF1F0200000084BE001103000000B1
:104278002864FF1F0200000086BE00110100000034
:10428800AC42FF1F02000000A0BD001101000000A9
:10429800C061FF1F0200000084BE0011030000007F
:1042A8002064FF1F120800000000000000C6C600BE
:1042B80000000000000000001311000000010000D1
:1042C80000000111FFFF00005048593600000000AF
:1042D800000000000B000500F0000000B4000028FA
:1042E800002800283075A000A000A000A000000849
:1042F8000008E001F000100010001000100010008D
:10430800100050005000500010001000D0070000AE
:10431800000000000F0001000500307507001000C4
:10432800010081FF00000000FF000000117400116F
:1043380019720011A96F0011FFFF0100FF000000B2
:104348002D9E0011A99B0011C19A001100000000C8
:104358000000000000000800040000003B00010805
:104368005902E00188212800FF0000000200000037
:104378008ABE00110100000050BF001102000000B9
:1043880086BE001101000000F143FF1F020000007B
:1043980082BE0011010000000068FF1F020000003B
:1043A80086BE001101000000F043FF1F020000005C
:1043B80080BE001101000000EE43FF1F0200000054
:1043C80086BE001101000000EC43FF1F0200000040
:1043D8007EBE001101000000E443FF1F1800180012
:1043E8001D0090010200000302020000020000000C
:1043F8008ABE00110100000064BF00110200000025
:1044080086BE0011010000003444FF1F02000000B6
:104418007CBE001100000000000000000200000047
:0E44280084BE0011030000002068FF1F20FF6B
:040000051FFF184180
:00000001FF
